
10_systick_delay.elf:     file format elf32-littlearm

Sections:
Idx Name          Size      VMA       LMA       File off  Algn
  0 .isr_vector   00000198  08000000  08000000  00010000  2**0
                  CONTENTS, ALLOC, LOAD, READONLY, DATA
  1 .text         0000137c  080001a0  080001a0  000101a0  2**4
                  CONTENTS, ALLOC, LOAD, READONLY, CODE
  2 .rodata       000000b0  0800151c  0800151c  0001151c  2**2
                  CONTENTS, ALLOC, LOAD, READONLY, DATA
  3 .ARM.extab    00000000  080015cc  080015cc  00020064  2**0
                  CONTENTS
  4 .ARM          00000000  080015cc  080015cc  00020064  2**0
                  CONTENTS
  5 .preinit_array 00000000  080015cc  080015cc  00020064  2**0
                  CONTENTS, ALLOC, LOAD, DATA
  6 .init_array   00000004  080015cc  080015cc  000115cc  2**2
                  CONTENTS, ALLOC, LOAD, DATA
  7 .fini_array   00000004  080015d0  080015d0  000115d0  2**2
                  CONTENTS, ALLOC, LOAD, DATA
  8 .data         00000064  20000000  080015d4  00020000  2**2
                  CONTENTS, ALLOC, LOAD, DATA
  9 .bss          00000038  20000064  08001638  00020064  2**2
                  ALLOC
 10 ._user_heap_stack 00000604  2000009c  08001638  0002009c  2**0
                  ALLOC
 11 .ARM.attributes 00000030  00000000  00000000  00020064  2**0
                  CONTENTS, READONLY
 12 .debug_info   00002d84  00000000  00000000  00020094  2**0
                  CONTENTS, READONLY, DEBUGGING, OCTETS
 13 .debug_abbrev 0000089b  00000000  00000000  00022e18  2**0
                  CONTENTS, READONLY, DEBUGGING, OCTETS
 14 .debug_aranges 00000180  00000000  00000000  000236b8  2**3
                  CONTENTS, READONLY, DEBUGGING, OCTETS
 15 .debug_ranges 00000128  00000000  00000000  00023838  2**3
                  CONTENTS, READONLY, DEBUGGING, OCTETS
 16 .debug_macro  00002005  00000000  00000000  00023960  2**0
                  CONTENTS, READONLY, DEBUGGING, OCTETS
 17 .debug_line   00001f0b  00000000  00000000  00025965  2**0
                  CONTENTS, READONLY, DEBUGGING, OCTETS
 18 .debug_str    00055392  00000000  00000000  00027870  2**0
                  CONTENTS, READONLY, DEBUGGING, OCTETS
 19 .comment      00000053  00000000  00000000  0007cc02  2**0
                  CONTENTS, READONLY
 20 .debug_frame  00000c50  00000000  00000000  0007cc58  2**2
                  CONTENTS, READONLY, DEBUGGING, OCTETS

Disassembly of section .text:

080001a0 <__do_global_dtors_aux>:
 80001a0:	b510      	push	{r4, lr}
 80001a2:	4c05      	ldr	r4, [pc, #20]	; (80001b8 <__do_global_dtors_aux+0x18>)
 80001a4:	7823      	ldrb	r3, [r4, #0]
 80001a6:	b933      	cbnz	r3, 80001b6 <__do_global_dtors_aux+0x16>
 80001a8:	4b04      	ldr	r3, [pc, #16]	; (80001bc <__do_global_dtors_aux+0x1c>)
 80001aa:	b113      	cbz	r3, 80001b2 <__do_global_dtors_aux+0x12>
 80001ac:	4804      	ldr	r0, [pc, #16]	; (80001c0 <__do_global_dtors_aux+0x20>)
 80001ae:	f3af 8000 	nop.w
 80001b2:	2301      	movs	r3, #1
 80001b4:	7023      	strb	r3, [r4, #0]
 80001b6:	bd10      	pop	{r4, pc}
 80001b8:	20000064 	.word	0x20000064
 80001bc:	00000000 	.word	0x00000000
 80001c0:	08001504 	.word	0x08001504

080001c4 <frame_dummy>:
 80001c4:	b508      	push	{r3, lr}
 80001c6:	4b03      	ldr	r3, [pc, #12]	; (80001d4 <frame_dummy+0x10>)
 80001c8:	b11b      	cbz	r3, 80001d2 <frame_dummy+0xe>
 80001ca:	4903      	ldr	r1, [pc, #12]	; (80001d8 <frame_dummy+0x14>)
 80001cc:	4803      	ldr	r0, [pc, #12]	; (80001dc <frame_dummy+0x18>)
 80001ce:	f3af 8000 	nop.w
 80001d2:	bd08      	pop	{r3, pc}
 80001d4:	00000000 	.word	0x00000000
 80001d8:	20000068 	.word	0x20000068
 80001dc:	08001504 	.word	0x08001504

080001e0 <memchr>:
 80001e0:	f001 01ff 	and.w	r1, r1, #255	; 0xff
 80001e4:	2a10      	cmp	r2, #16
 80001e6:	db2b      	blt.n	8000240 <memchr+0x60>
 80001e8:	f010 0f07 	tst.w	r0, #7
 80001ec:	d008      	beq.n	8000200 <memchr+0x20>
 80001ee:	f810 3b01 	ldrb.w	r3, [r0], #1
 80001f2:	3a01      	subs	r2, #1
 80001f4:	428b      	cmp	r3, r1
 80001f6:	d02d      	beq.n	8000254 <memchr+0x74>
 80001f8:	f010 0f07 	tst.w	r0, #7
 80001fc:	b342      	cbz	r2, 8000250 <memchr+0x70>
 80001fe:	d1f6      	bne.n	80001ee <memchr+0xe>
 8000200:	b4f0      	push	{r4, r5, r6, r7}
 8000202:	ea41 2101 	orr.w	r1, r1, r1, lsl #8
 8000206:	ea41 4101 	orr.w	r1, r1, r1, lsl #16
 800020a:	f022 0407 	bic.w	r4, r2, #7
 800020e:	f07f 0700 	mvns.w	r7, #0
 8000212:	2300      	movs	r3, #0
 8000214:	e8f0 5602 	ldrd	r5, r6, [r0], #8
 8000218:	3c08      	subs	r4, #8
 800021a:	ea85 0501 	eor.w	r5, r5, r1
 800021e:	ea86 0601 	eor.w	r6, r6, r1
 8000222:	fa85 f547 	uadd8	r5, r5, r7
 8000226:	faa3 f587 	sel	r5, r3, r7
 800022a:	fa86 f647 	uadd8	r6, r6, r7
 800022e:	faa5 f687 	sel	r6, r5, r7
 8000232:	b98e      	cbnz	r6, 8000258 <memchr+0x78>
 8000234:	d1ee      	bne.n	8000214 <memchr+0x34>
 8000236:	bcf0      	pop	{r4, r5, r6, r7}
 8000238:	f001 01ff 	and.w	r1, r1, #255	; 0xff
 800023c:	f002 0207 	and.w	r2, r2, #7
 8000240:	b132      	cbz	r2, 8000250 <memchr+0x70>
 8000242:	f810 3b01 	ldrb.w	r3, [r0], #1
 8000246:	3a01      	subs	r2, #1
 8000248:	ea83 0301 	eor.w	r3, r3, r1
 800024c:	b113      	cbz	r3, 8000254 <memchr+0x74>
 800024e:	d1f8      	bne.n	8000242 <memchr+0x62>
 8000250:	2000      	movs	r0, #0
 8000252:	4770      	bx	lr
 8000254:	3801      	subs	r0, #1
 8000256:	4770      	bx	lr
 8000258:	2d00      	cmp	r5, #0
 800025a:	bf06      	itte	eq
 800025c:	4635      	moveq	r5, r6
 800025e:	3803      	subeq	r0, #3
 8000260:	3807      	subne	r0, #7
 8000262:	f015 0f01 	tst.w	r5, #1
 8000266:	d107      	bne.n	8000278 <memchr+0x98>
 8000268:	3001      	adds	r0, #1
 800026a:	f415 7f80 	tst.w	r5, #256	; 0x100
 800026e:	bf02      	ittt	eq
 8000270:	3001      	addeq	r0, #1
 8000272:	f415 3fc0 	tsteq.w	r5, #98304	; 0x18000
 8000276:	3001      	addeq	r0, #1
 8000278:	bcf0      	pop	{r4, r5, r6, r7}
 800027a:	3801      	subs	r0, #1
 800027c:	4770      	bx	lr
 800027e:	bf00      	nop

08000280 <main>:
#define PIN_5		(1U<<5)
#define LED			PIN_5



int main(void){
 8000280:	b580      	push	{r7, lr}
 8000282:	af00      	add	r7, sp, #0

	RCC->AHB1ENR |= GPIOAEN;
 8000284:	4b10      	ldr	r3, [pc, #64]	; (80002c8 <main+0x48>)
 8000286:	6b1b      	ldr	r3, [r3, #48]	; 0x30
 8000288:	4a0f      	ldr	r2, [pc, #60]	; (80002c8 <main+0x48>)
 800028a:	f043 0301 	orr.w	r3, r3, #1
 800028e:	6313      	str	r3, [r2, #48]	; 0x30
	GPIOA->MODER |= (1U<<10);
 8000290:	4b0e      	ldr	r3, [pc, #56]	; (80002cc <main+0x4c>)
 8000292:	681b      	ldr	r3, [r3, #0]
 8000294:	4a0d      	ldr	r2, [pc, #52]	; (80002cc <main+0x4c>)
 8000296:	f443 6380 	orr.w	r3, r3, #1024	; 0x400
 800029a:	6013      	str	r3, [r2, #0]
	GPIOA->MODER &=~(1U<<11);
 800029c:	4b0b      	ldr	r3, [pc, #44]	; (80002cc <main+0x4c>)
 800029e:	681b      	ldr	r3, [r3, #0]
 80002a0:	4a0a      	ldr	r2, [pc, #40]	; (80002cc <main+0x4c>)
 80002a2:	f423 6300 	bic.w	r3, r3, #2048	; 0x800
 80002a6:	6013      	str	r3, [r2, #0]


	uart2_tx_init();
 80002a8:	f000 f8ee 	bl	8000488 <uart2_tx_init>

	while (1){
		printf("A Second passed!! \n\r");
 80002ac:	4808      	ldr	r0, [pc, #32]	; (80002d0 <main+0x50>)
 80002ae:	f000 f9d3 	bl	8000658 <iprintf>
		GPIOA->ODR ^=LED;
 80002b2:	4b06      	ldr	r3, [pc, #24]	; (80002cc <main+0x4c>)
 80002b4:	695b      	ldr	r3, [r3, #20]
 80002b6:	4a05      	ldr	r2, [pc, #20]	; (80002cc <main+0x4c>)
 80002b8:	f083 0320 	eor.w	r3, r3, #32
 80002bc:	6153      	str	r3, [r2, #20]
		systickDelayMs(1000);
 80002be:	f44f 707a 	mov.w	r0, #1000	; 0x3e8
 80002c2:	f000 f8ab 	bl	800041c <systickDelayMs>
		printf("A Second passed!! \n\r");
 80002c6:	e7f1      	b.n	80002ac <main+0x2c>
 80002c8:	40023800 	.word	0x40023800
 80002cc:	40020000 	.word	0x40020000
 80002d0:	0800151c 	.word	0x0800151c

080002d4 <_read>:
	_kill(status, -1);
	while (1) {}		/* Make sure we hang here */
}

__attribute__((weak)) int _read(int file, char *ptr, int len)
{
 80002d4:	b580      	push	{r7, lr}
 80002d6:	b086      	sub	sp, #24
 80002d8:	af00      	add	r7, sp, #0
 80002da:	60f8      	str	r0, [r7, #12]
 80002dc:	60b9      	str	r1, [r7, #8]
 80002de:	607a      	str	r2, [r7, #4]
	int DataIdx;

	for (DataIdx = 0; DataIdx < len; DataIdx++)
 80002e0:	2300      	movs	r3, #0
 80002e2:	617b      	str	r3, [r7, #20]
 80002e4:	e00a      	b.n	80002fc <_read+0x28>
	{
		*ptr++ = __io_getchar();
 80002e6:	f3af 8000 	nop.w
 80002ea:	4601      	mov	r1, r0
 80002ec:	68bb      	ldr	r3, [r7, #8]
 80002ee:	1c5a      	adds	r2, r3, #1
 80002f0:	60ba      	str	r2, [r7, #8]
 80002f2:	b2ca      	uxtb	r2, r1
 80002f4:	701a      	strb	r2, [r3, #0]
	for (DataIdx = 0; DataIdx < len; DataIdx++)
 80002f6:	697b      	ldr	r3, [r7, #20]
 80002f8:	3301      	adds	r3, #1
 80002fa:	617b      	str	r3, [r7, #20]
 80002fc:	697a      	ldr	r2, [r7, #20]
 80002fe:	687b      	ldr	r3, [r7, #4]
 8000300:	429a      	cmp	r2, r3
 8000302:	dbf0      	blt.n	80002e6 <_read+0x12>
	}

return len;
 8000304:	687b      	ldr	r3, [r7, #4]
}
 8000306:	4618      	mov	r0, r3
 8000308:	3718      	adds	r7, #24
 800030a:	46bd      	mov	sp, r7
 800030c:	bd80      	pop	{r7, pc}

0800030e <_write>:

__attribute__((weak)) int _write(int file, char *ptr, int len)
{
 800030e:	b580      	push	{r7, lr}
 8000310:	b086      	sub	sp, #24
 8000312:	af00      	add	r7, sp, #0
 8000314:	60f8      	str	r0, [r7, #12]
 8000316:	60b9      	str	r1, [r7, #8]
 8000318:	607a      	str	r2, [r7, #4]
	int DataIdx;

	for (DataIdx = 0; DataIdx < len; DataIdx++)
 800031a:	2300      	movs	r3, #0
 800031c:	617b      	str	r3, [r7, #20]
 800031e:	e009      	b.n	8000334 <_write+0x26>
	{
		__io_putchar(*ptr++);
 8000320:	68bb      	ldr	r3, [r7, #8]
 8000322:	1c5a      	adds	r2, r3, #1
 8000324:	60ba      	str	r2, [r7, #8]
 8000326:	781b      	ldrb	r3, [r3, #0]
 8000328:	4618      	mov	r0, r3
 800032a:	f000 f8a1 	bl	8000470 <__io_putchar>
	for (DataIdx = 0; DataIdx < len; DataIdx++)
 800032e:	697b      	ldr	r3, [r7, #20]
 8000330:	3301      	adds	r3, #1
 8000332:	617b      	str	r3, [r7, #20]
 8000334:	697a      	ldr	r2, [r7, #20]
 8000336:	687b      	ldr	r3, [r7, #4]
 8000338:	429a      	cmp	r2, r3
 800033a:	dbf1      	blt.n	8000320 <_write+0x12>
	}
	return len;
 800033c:	687b      	ldr	r3, [r7, #4]
}
 800033e:	4618      	mov	r0, r3
 8000340:	3718      	adds	r7, #24
 8000342:	46bd      	mov	sp, r7
 8000344:	bd80      	pop	{r7, pc}

08000346 <_close>:

int _close(int file)
{
 8000346:	b480      	push	{r7}
 8000348:	b083      	sub	sp, #12
 800034a:	af00      	add	r7, sp, #0
 800034c:	6078      	str	r0, [r7, #4]
	return -1;
 800034e:	f04f 33ff 	mov.w	r3, #4294967295
}
 8000352:	4618      	mov	r0, r3
 8000354:	370c      	adds	r7, #12
 8000356:	46bd      	mov	sp, r7
 8000358:	f85d 7b04 	ldr.w	r7, [sp], #4
 800035c:	4770      	bx	lr

0800035e <_fstat>:


int _fstat(int file, struct stat *st)
{
 800035e:	b480      	push	{r7}
 8000360:	b083      	sub	sp, #12
 8000362:	af00      	add	r7, sp, #0
 8000364:	6078      	str	r0, [r7, #4]
 8000366:	6039      	str	r1, [r7, #0]
	st->st_mode = S_IFCHR;
 8000368:	683b      	ldr	r3, [r7, #0]
 800036a:	f44f 5200 	mov.w	r2, #8192	; 0x2000
 800036e:	605a      	str	r2, [r3, #4]
	return 0;
 8000370:	2300      	movs	r3, #0
}
 8000372:	4618      	mov	r0, r3
 8000374:	370c      	adds	r7, #12
 8000376:	46bd      	mov	sp, r7
 8000378:	f85d 7b04 	ldr.w	r7, [sp], #4
 800037c:	4770      	bx	lr

0800037e <_isatty>:

int _isatty(int file)
{
 800037e:	b480      	push	{r7}
 8000380:	b083      	sub	sp, #12
 8000382:	af00      	add	r7, sp, #0
 8000384:	6078      	str	r0, [r7, #4]
	return 1;
 8000386:	2301      	movs	r3, #1
}
 8000388:	4618      	mov	r0, r3
 800038a:	370c      	adds	r7, #12
 800038c:	46bd      	mov	sp, r7
 800038e:	f85d 7b04 	ldr.w	r7, [sp], #4
 8000392:	4770      	bx	lr

08000394 <_lseek>:

int _lseek(int file, int ptr, int dir)
{
 8000394:	b480      	push	{r7}
 8000396:	b085      	sub	sp, #20
 8000398:	af00      	add	r7, sp, #0
 800039a:	60f8      	str	r0, [r7, #12]
 800039c:	60b9      	str	r1, [r7, #8]
 800039e:	607a      	str	r2, [r7, #4]
	return 0;
 80003a0:	2300      	movs	r3, #0
}
 80003a2:	4618      	mov	r0, r3
 80003a4:	3714      	adds	r7, #20
 80003a6:	46bd      	mov	sp, r7
 80003a8:	f85d 7b04 	ldr.w	r7, [sp], #4
 80003ac:	4770      	bx	lr
	...

080003b0 <_sbrk>:
 *
 * @param incr Memory size
 * @return Pointer to allocated memory
 */
void *_sbrk(ptrdiff_t incr)
{
 80003b0:	b580      	push	{r7, lr}
 80003b2:	b086      	sub	sp, #24
 80003b4:	af00      	add	r7, sp, #0
 80003b6:	6078      	str	r0, [r7, #4]
  extern uint8_t _end; /* Symbol defined in the linker script */
  extern uint8_t _estack; /* Symbol defined in the linker script */
  extern uint32_t _Min_Stack_Size; /* Symbol defined in the linker script */
  const uint32_t stack_limit = (uint32_t)&_estack - (uint32_t)&_Min_Stack_Size;
 80003b8:	4a14      	ldr	r2, [pc, #80]	; (800040c <_sbrk+0x5c>)
 80003ba:	4b15      	ldr	r3, [pc, #84]	; (8000410 <_sbrk+0x60>)
 80003bc:	1ad3      	subs	r3, r2, r3
 80003be:	617b      	str	r3, [r7, #20]
  const uint8_t *max_heap = (uint8_t *)stack_limit;
 80003c0:	697b      	ldr	r3, [r7, #20]
 80003c2:	613b      	str	r3, [r7, #16]
  uint8_t *prev_heap_end;

  /* Initialize heap end at first call */
  if (NULL == __sbrk_heap_end)
 80003c4:	4b13      	ldr	r3, [pc, #76]	; (8000414 <_sbrk+0x64>)
 80003c6:	681b      	ldr	r3, [r3, #0]
 80003c8:	2b00      	cmp	r3, #0
 80003ca:	d102      	bne.n	80003d2 <_sbrk+0x22>
  {
    __sbrk_heap_end = &_end;
 80003cc:	4b11      	ldr	r3, [pc, #68]	; (8000414 <_sbrk+0x64>)
 80003ce:	4a12      	ldr	r2, [pc, #72]	; (8000418 <_sbrk+0x68>)
 80003d0:	601a      	str	r2, [r3, #0]
  }

  /* Protect heap from growing into the reserved MSP stack */
  if (__sbrk_heap_end + incr > max_heap)
 80003d2:	4b10      	ldr	r3, [pc, #64]	; (8000414 <_sbrk+0x64>)
 80003d4:	681a      	ldr	r2, [r3, #0]
 80003d6:	687b      	ldr	r3, [r7, #4]
 80003d8:	4413      	add	r3, r2
 80003da:	693a      	ldr	r2, [r7, #16]
 80003dc:	429a      	cmp	r2, r3
 80003de:	d207      	bcs.n	80003f0 <_sbrk+0x40>
  {
    errno = ENOMEM;
 80003e0:	f000 f908 	bl	80005f4 <__errno>
 80003e4:	4603      	mov	r3, r0
 80003e6:	220c      	movs	r2, #12
 80003e8:	601a      	str	r2, [r3, #0]
    return (void *)-1;
 80003ea:	f04f 33ff 	mov.w	r3, #4294967295
 80003ee:	e009      	b.n	8000404 <_sbrk+0x54>
  }

  prev_heap_end = __sbrk_heap_end;
 80003f0:	4b08      	ldr	r3, [pc, #32]	; (8000414 <_sbrk+0x64>)
 80003f2:	681b      	ldr	r3, [r3, #0]
 80003f4:	60fb      	str	r3, [r7, #12]
  __sbrk_heap_end += incr;
 80003f6:	4b07      	ldr	r3, [pc, #28]	; (8000414 <_sbrk+0x64>)
 80003f8:	681a      	ldr	r2, [r3, #0]
 80003fa:	687b      	ldr	r3, [r7, #4]
 80003fc:	4413      	add	r3, r2
 80003fe:	4a05      	ldr	r2, [pc, #20]	; (8000414 <_sbrk+0x64>)
 8000400:	6013      	str	r3, [r2, #0]

  return (void *)prev_heap_end;
 8000402:	68fb      	ldr	r3, [r7, #12]
}
 8000404:	4618      	mov	r0, r3
 8000406:	3718      	adds	r7, #24
 8000408:	46bd      	mov	sp, r7
 800040a:	bd80      	pop	{r7, pc}
 800040c:	20020000 	.word	0x20020000
 8000410:	00000400 	.word	0x00000400
 8000414:	20000080 	.word	0x20000080
 8000418:	200000a0 	.word	0x200000a0

0800041c <systickDelayMs>:
#define CTRL_CLKSRC			(1U<<2)
#define CTRL_COUNTFLAG 		(1U<<16)



void systickDelayMs(int delay){
 800041c:	b480      	push	{r7}
 800041e:	b085      	sub	sp, #20
 8000420:	af00      	add	r7, sp, #0
 8000422:	6078      	str	r0, [r7, #4]
	/*reload with number of clocks per millisecond*/
	SysTick->LOAD = SYSTICK_LOAD_VAL;
 8000424:	4b11      	ldr	r3, [pc, #68]	; (800046c <systickDelayMs+0x50>)
 8000426:	f44f 527a 	mov.w	r2, #16000	; 0x3e80
 800042a:	605a      	str	r2, [r3, #4]

	/*clear systick current value register*/
	SysTick->VAL = 0;
 800042c:	4b0f      	ldr	r3, [pc, #60]	; (800046c <systickDelayMs+0x50>)
 800042e:	2200      	movs	r2, #0
 8000430:	609a      	str	r2, [r3, #8]

	/*enable systick and select internal clk src*/
	SysTick->CTRL = CTRL_ENABLE | CTRL_CLKSRC;
 8000432:	4b0e      	ldr	r3, [pc, #56]	; (800046c <systickDelayMs+0x50>)
 8000434:	2205      	movs	r2, #5
 8000436:	601a      	str	r2, [r3, #0]
	/**/
	/**/
	for(int i=0; i< delay; i++){
 8000438:	2300      	movs	r3, #0
 800043a:	60fb      	str	r3, [r7, #12]
 800043c:	e009      	b.n	8000452 <systickDelayMs+0x36>
		/*wait until the COUNTFLAG is set*/
		while((SysTick->CTRL & CTRL_COUNTFLAG) == 0){}
 800043e:	bf00      	nop
 8000440:	4b0a      	ldr	r3, [pc, #40]	; (800046c <systickDelayMs+0x50>)
 8000442:	681b      	ldr	r3, [r3, #0]
 8000444:	f403 3380 	and.w	r3, r3, #65536	; 0x10000
 8000448:	2b00      	cmp	r3, #0
 800044a:	d0f9      	beq.n	8000440 <systickDelayMs+0x24>
	for(int i=0; i< delay; i++){
 800044c:	68fb      	ldr	r3, [r7, #12]
 800044e:	3301      	adds	r3, #1
 8000450:	60fb      	str	r3, [r7, #12]
 8000452:	68fa      	ldr	r2, [r7, #12]
 8000454:	687b      	ldr	r3, [r7, #4]
 8000456:	429a      	cmp	r2, r3
 8000458:	dbf1      	blt.n	800043e <systickDelayMs+0x22>
	}
	SysTick->CTRL = 0;
 800045a:	4b04      	ldr	r3, [pc, #16]	; (800046c <systickDelayMs+0x50>)
 800045c:	2200      	movs	r2, #0
 800045e:	601a      	str	r2, [r3, #0]

}
 8000460:	bf00      	nop
 8000462:	3714      	adds	r7, #20
 8000464:	46bd      	mov	sp, r7
 8000466:	f85d 7b04 	ldr.w	r7, [sp], #4
 800046a:	4770      	bx	lr
 800046c:	e000e010 	.word	0xe000e010

08000470 <__io_putchar>:



void uart2_write(int ch);

int __io_putchar(int ch){
 8000470:	b580      	push	{r7, lr}
 8000472:	b082      	sub	sp, #8
 8000474:	af00      	add	r7, sp, #0
 8000476:	6078      	str	r0, [r7, #4]
	uart2_write(ch);
 8000478:	6878      	ldr	r0, [r7, #4]
 800047a:	f000 f853 	bl	8000524 <uart2_write>
	return ch;
 800047e:	687b      	ldr	r3, [r7, #4]
}
 8000480:	4618      	mov	r0, r3
 8000482:	3708      	adds	r7, #8
 8000484:	46bd      	mov	sp, r7
 8000486:	bd80      	pop	{r7, pc}

08000488 <uart2_tx_init>:

void uart2_tx_init(void){
 8000488:	b580      	push	{r7, lr}
 800048a:	af00      	add	r7, sp, #0
	/*********configure the uart gpioa pin*********/
	/*enable clock access to gpioa*/
	RCC->AHB1ENR |= GPIOAEN;
 800048c:	4b21      	ldr	r3, [pc, #132]	; (8000514 <uart2_tx_init+0x8c>)
 800048e:	6b1b      	ldr	r3, [r3, #48]	; 0x30
 8000490:	4a20      	ldr	r2, [pc, #128]	; (8000514 <uart2_tx_init+0x8c>)
 8000492:	f043 0301 	orr.w	r3, r3, #1
 8000496:	6313      	str	r3, [r2, #48]	; 0x30

	/*set PA2 mode to alternate function mode*/
	GPIOA->MODER &= ~(1U<<4);
 8000498:	4b1f      	ldr	r3, [pc, #124]	; (8000518 <uart2_tx_init+0x90>)
 800049a:	681b      	ldr	r3, [r3, #0]
 800049c:	4a1e      	ldr	r2, [pc, #120]	; (8000518 <uart2_tx_init+0x90>)
 800049e:	f023 0310 	bic.w	r3, r3, #16
 80004a2:	6013      	str	r3, [r2, #0]
	GPIOA->MODER |= (1U<<5);
 80004a4:	4b1c      	ldr	r3, [pc, #112]	; (8000518 <uart2_tx_init+0x90>)
 80004a6:	681b      	ldr	r3, [r3, #0]
 80004a8:	4a1b      	ldr	r2, [pc, #108]	; (8000518 <uart2_tx_init+0x90>)
 80004aa:	f043 0320 	orr.w	r3, r3, #32
 80004ae:	6013      	str	r3, [r2, #0]

	/*set PA2 alternate function type to UART_TX (AF07)*/
	GPIOA->AFR[0] |= (1U<<8);
 80004b0:	4b19      	ldr	r3, [pc, #100]	; (8000518 <uart2_tx_init+0x90>)
 80004b2:	6a1b      	ldr	r3, [r3, #32]
 80004b4:	4a18      	ldr	r2, [pc, #96]	; (8000518 <uart2_tx_init+0x90>)
 80004b6:	f443 7380 	orr.w	r3, r3, #256	; 0x100
 80004ba:	6213      	str	r3, [r2, #32]
	GPIOA->AFR[0] |= (1U<<9);
 80004bc:	4b16      	ldr	r3, [pc, #88]	; (8000518 <uart2_tx_init+0x90>)
 80004be:	6a1b      	ldr	r3, [r3, #32]
 80004c0:	4a15      	ldr	r2, [pc, #84]	; (8000518 <uart2_tx_init+0x90>)
 80004c2:	f443 7300 	orr.w	r3, r3, #512	; 0x200
 80004c6:	6213      	str	r3, [r2, #32]
	GPIOA->AFR[0] |= (1U<<10);
 80004c8:	4b13      	ldr	r3, [pc, #76]	; (8000518 <uart2_tx_init+0x90>)
 80004ca:	6a1b      	ldr	r3, [r3, #32]
 80004cc:	4a12      	ldr	r2, [pc, #72]	; (8000518 <uart2_tx_init+0x90>)
 80004ce:	f443 6380 	orr.w	r3, r3, #1024	; 0x400
 80004d2:	6213      	str	r3, [r2, #32]
	GPIOA->AFR[0] &= ~(1U<<11);
 80004d4:	4b10      	ldr	r3, [pc, #64]	; (8000518 <uart2_tx_init+0x90>)
 80004d6:	6a1b      	ldr	r3, [r3, #32]
 80004d8:	4a0f      	ldr	r2, [pc, #60]	; (8000518 <uart2_tx_init+0x90>)
 80004da:	f423 6300 	bic.w	r3, r3, #2048	; 0x800
 80004de:	6213      	str	r3, [r2, #32]

	/*********configure the uart module *********/
	/*enable clock access to uart2*/
	RCC->APB1ENR |= UART2EN;
 80004e0:	4b0c      	ldr	r3, [pc, #48]	; (8000514 <uart2_tx_init+0x8c>)
 80004e2:	6c1b      	ldr	r3, [r3, #64]	; 0x40
 80004e4:	4a0b      	ldr	r2, [pc, #44]	; (8000514 <uart2_tx_init+0x8c>)
 80004e6:	f443 3300 	orr.w	r3, r3, #131072	; 0x20000
 80004ea:	6413      	str	r3, [r2, #64]	; 0x40

	/*configure baudrate*/
	uart_set_baudrate(USART2,APB1_CLK,UART_BAUDRATE);
 80004ec:	f44f 32e1 	mov.w	r2, #115200	; 0x1c200
 80004f0:	490a      	ldr	r1, [pc, #40]	; (800051c <uart2_tx_init+0x94>)
 80004f2:	480b      	ldr	r0, [pc, #44]	; (8000520 <uart2_tx_init+0x98>)
 80004f4:	f000 f82e 	bl	8000554 <uart_set_baudrate>

	/*configure the transfer direction*/
	USART2 ->CR1 |= CR1_TE;
 80004f8:	4b09      	ldr	r3, [pc, #36]	; (8000520 <uart2_tx_init+0x98>)
 80004fa:	68db      	ldr	r3, [r3, #12]
 80004fc:	4a08      	ldr	r2, [pc, #32]	; (8000520 <uart2_tx_init+0x98>)
 80004fe:	f043 0308 	orr.w	r3, r3, #8
 8000502:	60d3      	str	r3, [r2, #12]

	/*enable uart module*/
	USART2 ->CR1 |= CR1_UE;
 8000504:	4b06      	ldr	r3, [pc, #24]	; (8000520 <uart2_tx_init+0x98>)
 8000506:	68db      	ldr	r3, [r3, #12]
 8000508:	4a05      	ldr	r2, [pc, #20]	; (8000520 <uart2_tx_init+0x98>)
 800050a:	f443 5300 	orr.w	r3, r3, #8192	; 0x2000
 800050e:	60d3      	str	r3, [r2, #12]

}
 8000510:	bf00      	nop
 8000512:	bd80      	pop	{r7, pc}
 8000514:	40023800 	.word	0x40023800
 8000518:	40020000 	.word	0x40020000
 800051c:	00f42400 	.word	0x00f42400
 8000520:	40004400 	.word	0x40004400

08000524 <uart2_write>:
	while(!(USART2->SR & SR_RXE)){}
	/*write to transmit data register*/
	return USART2->DR;
}

void uart2_write(int ch){
 8000524:	b480      	push	{r7}
 8000526:	b083      	sub	sp, #12
 8000528:	af00      	add	r7, sp, #0
 800052a:	6078      	str	r0, [r7, #4]
	/*make sure the transmit data register is empty*/
	while(!(USART2->SR & SR_TXE)){}
 800052c:	bf00      	nop
 800052e:	4b08      	ldr	r3, [pc, #32]	; (8000550 <uart2_write+0x2c>)
 8000530:	681b      	ldr	r3, [r3, #0]
 8000532:	f003 0380 	and.w	r3, r3, #128	; 0x80
 8000536:	2b00      	cmp	r3, #0
 8000538:	d0f9      	beq.n	800052e <uart2_write+0xa>
	/*write to transmit data register*/
	USART2->DR = (ch & 0xFF);
 800053a:	687b      	ldr	r3, [r7, #4]
 800053c:	4a04      	ldr	r2, [pc, #16]	; (8000550 <uart2_write+0x2c>)
 800053e:	b2db      	uxtb	r3, r3
 8000540:	6053      	str	r3, [r2, #4]
}
 8000542:	bf00      	nop
 8000544:	370c      	adds	r7, #12
 8000546:	46bd      	mov	sp, r7
 8000548:	f85d 7b04 	ldr.w	r7, [sp], #4
 800054c:	4770      	bx	lr
 800054e:	bf00      	nop
 8000550:	40004400 	.word	0x40004400

08000554 <uart_set_baudrate>:

static void uart_set_baudrate(USART_TypeDef *USARTx, uint32_t PeriphClk, uint32_t BaudRate){
 8000554:	b580      	push	{r7, lr}
 8000556:	b084      	sub	sp, #16
 8000558:	af00      	add	r7, sp, #0
 800055a:	60f8      	str	r0, [r7, #12]
 800055c:	60b9      	str	r1, [r7, #8]
 800055e:	607a      	str	r2, [r7, #4]
	USARTx->BRR = compute_uart_bd(PeriphClk, BaudRate);
 8000560:	6879      	ldr	r1, [r7, #4]
 8000562:	68b8      	ldr	r0, [r7, #8]
 8000564:	f000 f808 	bl	8000578 <compute_uart_bd>
 8000568:	4603      	mov	r3, r0
 800056a:	461a      	mov	r2, r3
 800056c:	68fb      	ldr	r3, [r7, #12]
 800056e:	609a      	str	r2, [r3, #8]
}
 8000570:	bf00      	nop
 8000572:	3710      	adds	r7, #16
 8000574:	46bd      	mov	sp, r7
 8000576:	bd80      	pop	{r7, pc}

08000578 <compute_uart_bd>:

static uint16_t compute_uart_bd(uint32_t PeriphClk, uint32_t BaudRate){
 8000578:	b480      	push	{r7}
 800057a:	b083      	sub	sp, #12
 800057c:	af00      	add	r7, sp, #0
 800057e:	6078      	str	r0, [r7, #4]
 8000580:	6039      	str	r1, [r7, #0]
	return ((PeriphClk + (BaudRate/2U))/BaudRate);
 8000582:	683b      	ldr	r3, [r7, #0]
 8000584:	085a      	lsrs	r2, r3, #1
 8000586:	687b      	ldr	r3, [r7, #4]
 8000588:	441a      	add	r2, r3
 800058a:	683b      	ldr	r3, [r7, #0]
 800058c:	fbb2 f3f3 	udiv	r3, r2, r3
 8000590:	b29b      	uxth	r3, r3
}
 8000592:	4618      	mov	r0, r3
 8000594:	370c      	adds	r7, #12
 8000596:	46bd      	mov	sp, r7
 8000598:	f85d 7b04 	ldr.w	r7, [sp], #4
 800059c:	4770      	bx	lr
	...

080005a0 <Reset_Handler>:

  .section .text.Reset_Handler
  .weak Reset_Handler
  .type Reset_Handler, %function
Reset_Handler:
  ldr   r0, =_estack
 80005a0:	480d      	ldr	r0, [pc, #52]	; (80005d8 <LoopForever+0x2>)
  mov   sp, r0          /* set stack pointer */
 80005a2:	4685      	mov	sp, r0
/* Call the clock system intitialization function.*/
  bl  SystemInit
 80005a4:	f3af 8000 	nop.w

/* Copy the data segment initializers from flash to SRAM */
  ldr r0, =_sdata
 80005a8:	480c      	ldr	r0, [pc, #48]	; (80005dc <LoopForever+0x6>)
  ldr r1, =_edata
 80005aa:	490d      	ldr	r1, [pc, #52]	; (80005e0 <LoopForever+0xa>)
  ldr r2, =_sidata
 80005ac:	4a0d      	ldr	r2, [pc, #52]	; (80005e4 <LoopForever+0xe>)
  movs r3, #0
 80005ae:	2300      	movs	r3, #0
  b LoopCopyDataInit
 80005b0:	e002      	b.n	80005b8 <LoopCopyDataInit>

080005b2 <CopyDataInit>:

CopyDataInit:
  ldr r4, [r2, r3]
 80005b2:	58d4      	ldr	r4, [r2, r3]
  str r4, [r0, r3]
 80005b4:	50c4      	str	r4, [r0, r3]
  adds r3, r3, #4
 80005b6:	3304      	adds	r3, #4

080005b8 <LoopCopyDataInit>:

LoopCopyDataInit:
  adds r4, r0, r3
 80005b8:	18c4      	adds	r4, r0, r3
  cmp r4, r1
 80005ba:	428c      	cmp	r4, r1
  bcc CopyDataInit
 80005bc:	d3f9      	bcc.n	80005b2 <CopyDataInit>

/* Zero fill the bss segment. */
  ldr r2, =_sbss
 80005be:	4a0a      	ldr	r2, [pc, #40]	; (80005e8 <LoopForever+0x12>)
  ldr r4, =_ebss
 80005c0:	4c0a      	ldr	r4, [pc, #40]	; (80005ec <LoopForever+0x16>)
  movs r3, #0
 80005c2:	2300      	movs	r3, #0
  b LoopFillZerobss
 80005c4:	e001      	b.n	80005ca <LoopFillZerobss>

080005c6 <FillZerobss>:

FillZerobss:
  str  r3, [r2]
 80005c6:	6013      	str	r3, [r2, #0]
  adds r2, r2, #4
 80005c8:	3204      	adds	r2, #4

080005ca <LoopFillZerobss>:

LoopFillZerobss:
  cmp r2, r4
 80005ca:	42a2      	cmp	r2, r4
  bcc FillZerobss
 80005cc:	d3fb      	bcc.n	80005c6 <FillZerobss>

/* Call static constructors */
  bl __libc_init_array
 80005ce:	f000 f817 	bl	8000600 <__libc_init_array>
/* Call the application's entry point.*/
  bl main
 80005d2:	f7ff fe55 	bl	8000280 <main>

080005d6 <LoopForever>:

LoopForever:
    b LoopForever
 80005d6:	e7fe      	b.n	80005d6 <LoopForever>
  ldr   r0, =_estack
 80005d8:	20020000 	.word	0x20020000
  ldr r0, =_sdata
 80005dc:	20000000 	.word	0x20000000
  ldr r1, =_edata
 80005e0:	20000064 	.word	0x20000064
  ldr r2, =_sidata
 80005e4:	080015d4 	.word	0x080015d4
  ldr r2, =_sbss
 80005e8:	20000064 	.word	0x20000064
  ldr r4, =_ebss
 80005ec:	2000009c 	.word	0x2000009c

080005f0 <ADC_IRQHandler>:
 * @retval : None
*/
  .section .text.Default_Handler,"ax",%progbits
Default_Handler:
Infinite_Loop:
  b Infinite_Loop
 80005f0:	e7fe      	b.n	80005f0 <ADC_IRQHandler>
	...

080005f4 <__errno>:
 80005f4:	4b01      	ldr	r3, [pc, #4]	; (80005fc <__errno+0x8>)
 80005f6:	6818      	ldr	r0, [r3, #0]
 80005f8:	4770      	bx	lr
 80005fa:	bf00      	nop
 80005fc:	20000000 	.word	0x20000000

08000600 <__libc_init_array>:
 8000600:	b570      	push	{r4, r5, r6, lr}
 8000602:	4d0d      	ldr	r5, [pc, #52]	; (8000638 <__libc_init_array+0x38>)
 8000604:	4c0d      	ldr	r4, [pc, #52]	; (800063c <__libc_init_array+0x3c>)
 8000606:	1b64      	subs	r4, r4, r5
 8000608:	10a4      	asrs	r4, r4, #2
 800060a:	2600      	movs	r6, #0
 800060c:	42a6      	cmp	r6, r4
 800060e:	d109      	bne.n	8000624 <__libc_init_array+0x24>
 8000610:	4d0b      	ldr	r5, [pc, #44]	; (8000640 <__libc_init_array+0x40>)
 8000612:	4c0c      	ldr	r4, [pc, #48]	; (8000644 <__libc_init_array+0x44>)
 8000614:	f000 ff76 	bl	8001504 <_init>
 8000618:	1b64      	subs	r4, r4, r5
 800061a:	10a4      	asrs	r4, r4, #2
 800061c:	2600      	movs	r6, #0
 800061e:	42a6      	cmp	r6, r4
 8000620:	d105      	bne.n	800062e <__libc_init_array+0x2e>
 8000622:	bd70      	pop	{r4, r5, r6, pc}
 8000624:	f855 3b04 	ldr.w	r3, [r5], #4
 8000628:	4798      	blx	r3
 800062a:	3601      	adds	r6, #1
 800062c:	e7ee      	b.n	800060c <__libc_init_array+0xc>
 800062e:	f855 3b04 	ldr.w	r3, [r5], #4
 8000632:	4798      	blx	r3
 8000634:	3601      	adds	r6, #1
 8000636:	e7f2      	b.n	800061e <__libc_init_array+0x1e>
 8000638:	080015cc 	.word	0x080015cc
 800063c:	080015cc 	.word	0x080015cc
 8000640:	080015cc 	.word	0x080015cc
 8000644:	080015d0 	.word	0x080015d0

08000648 <memset>:
 8000648:	4402      	add	r2, r0
 800064a:	4603      	mov	r3, r0
 800064c:	4293      	cmp	r3, r2
 800064e:	d100      	bne.n	8000652 <memset+0xa>
 8000650:	4770      	bx	lr
 8000652:	f803 1b01 	strb.w	r1, [r3], #1
 8000656:	e7f9      	b.n	800064c <memset+0x4>

08000658 <iprintf>:
 8000658:	b40f      	push	{r0, r1, r2, r3}
 800065a:	4b0a      	ldr	r3, [pc, #40]	; (8000684 <iprintf+0x2c>)
 800065c:	b513      	push	{r0, r1, r4, lr}
 800065e:	681c      	ldr	r4, [r3, #0]
 8000660:	b124      	cbz	r4, 800066c <iprintf+0x14>
 8000662:	69a3      	ldr	r3, [r4, #24]
 8000664:	b913      	cbnz	r3, 800066c <iprintf+0x14>
 8000666:	4620      	mov	r0, r4
 8000668:	f000 f866 	bl	8000738 <__sinit>
 800066c:	ab05      	add	r3, sp, #20
 800066e:	9a04      	ldr	r2, [sp, #16]
 8000670:	68a1      	ldr	r1, [r4, #8]
 8000672:	9301      	str	r3, [sp, #4]
 8000674:	4620      	mov	r0, r4
 8000676:	f000 f983 	bl	8000980 <_vfiprintf_r>
 800067a:	b002      	add	sp, #8
 800067c:	e8bd 4010 	ldmia.w	sp!, {r4, lr}
 8000680:	b004      	add	sp, #16
 8000682:	4770      	bx	lr
 8000684:	20000000 	.word	0x20000000

08000688 <std>:
 8000688:	2300      	movs	r3, #0
 800068a:	b510      	push	{r4, lr}
 800068c:	4604      	mov	r4, r0
 800068e:	e9c0 3300 	strd	r3, r3, [r0]
 8000692:	e9c0 3304 	strd	r3, r3, [r0, #16]
 8000696:	6083      	str	r3, [r0, #8]
 8000698:	8181      	strh	r1, [r0, #12]
 800069a:	6643      	str	r3, [r0, #100]	; 0x64
 800069c:	81c2      	strh	r2, [r0, #14]
 800069e:	6183      	str	r3, [r0, #24]
 80006a0:	4619      	mov	r1, r3
 80006a2:	2208      	movs	r2, #8
 80006a4:	305c      	adds	r0, #92	; 0x5c
 80006a6:	f7ff ffcf 	bl	8000648 <memset>
 80006aa:	4b05      	ldr	r3, [pc, #20]	; (80006c0 <std+0x38>)
 80006ac:	6263      	str	r3, [r4, #36]	; 0x24
 80006ae:	4b05      	ldr	r3, [pc, #20]	; (80006c4 <std+0x3c>)
 80006b0:	62a3      	str	r3, [r4, #40]	; 0x28
 80006b2:	4b05      	ldr	r3, [pc, #20]	; (80006c8 <std+0x40>)
 80006b4:	62e3      	str	r3, [r4, #44]	; 0x2c
 80006b6:	4b05      	ldr	r3, [pc, #20]	; (80006cc <std+0x44>)
 80006b8:	6224      	str	r4, [r4, #32]
 80006ba:	6323      	str	r3, [r4, #48]	; 0x30
 80006bc:	bd10      	pop	{r4, pc}
 80006be:	bf00      	nop
 80006c0:	08000f29 	.word	0x08000f29
 80006c4:	08000f4b 	.word	0x08000f4b
 80006c8:	08000f83 	.word	0x08000f83
 80006cc:	08000fa7 	.word	0x08000fa7

080006d0 <_cleanup_r>:
 80006d0:	4901      	ldr	r1, [pc, #4]	; (80006d8 <_cleanup_r+0x8>)
 80006d2:	f000 b8af 	b.w	8000834 <_fwalk_reent>
 80006d6:	bf00      	nop
 80006d8:	08001281 	.word	0x08001281

080006dc <__sfmoreglue>:
 80006dc:	b570      	push	{r4, r5, r6, lr}
 80006de:	1e4a      	subs	r2, r1, #1
 80006e0:	2568      	movs	r5, #104	; 0x68
 80006e2:	4355      	muls	r5, r2
 80006e4:	460e      	mov	r6, r1
 80006e6:	f105 0174 	add.w	r1, r5, #116	; 0x74
 80006ea:	f000 f8c5 	bl	8000878 <_malloc_r>
 80006ee:	4604      	mov	r4, r0
 80006f0:	b140      	cbz	r0, 8000704 <__sfmoreglue+0x28>
 80006f2:	2100      	movs	r1, #0
 80006f4:	e9c0 1600 	strd	r1, r6, [r0]
 80006f8:	300c      	adds	r0, #12
 80006fa:	60a0      	str	r0, [r4, #8]
 80006fc:	f105 0268 	add.w	r2, r5, #104	; 0x68
 8000700:	f7ff ffa2 	bl	8000648 <memset>
 8000704:	4620      	mov	r0, r4
 8000706:	bd70      	pop	{r4, r5, r6, pc}

08000708 <__sfp_lock_acquire>:
 8000708:	4801      	ldr	r0, [pc, #4]	; (8000710 <__sfp_lock_acquire+0x8>)
 800070a:	f000 b8b3 	b.w	8000874 <__retarget_lock_acquire_recursive>
 800070e:	bf00      	nop
 8000710:	20000094 	.word	0x20000094

08000714 <__sfp_lock_release>:
 8000714:	4801      	ldr	r0, [pc, #4]	; (800071c <__sfp_lock_release+0x8>)
 8000716:	f000 b8ae 	b.w	8000876 <__retarget_lock_release_recursive>
 800071a:	bf00      	nop
 800071c:	20000094 	.word	0x20000094

08000720 <__sinit_lock_acquire>:
 8000720:	4801      	ldr	r0, [pc, #4]	; (8000728 <__sinit_lock_acquire+0x8>)
 8000722:	f000 b8a7 	b.w	8000874 <__retarget_lock_acquire_recursive>
 8000726:	bf00      	nop
 8000728:	2000008f 	.word	0x2000008f

0800072c <__sinit_lock_release>:
 800072c:	4801      	ldr	r0, [pc, #4]	; (8000734 <__sinit_lock_release+0x8>)
 800072e:	f000 b8a2 	b.w	8000876 <__retarget_lock_release_recursive>
 8000732:	bf00      	nop
 8000734:	2000008f 	.word	0x2000008f

08000738 <__sinit>:
 8000738:	b510      	push	{r4, lr}
 800073a:	4604      	mov	r4, r0
 800073c:	f7ff fff0 	bl	8000720 <__sinit_lock_acquire>
 8000740:	69a3      	ldr	r3, [r4, #24]
 8000742:	b11b      	cbz	r3, 800074c <__sinit+0x14>
 8000744:	e8bd 4010 	ldmia.w	sp!, {r4, lr}
 8000748:	f7ff bff0 	b.w	800072c <__sinit_lock_release>
 800074c:	e9c4 3312 	strd	r3, r3, [r4, #72]	; 0x48
 8000750:	6523      	str	r3, [r4, #80]	; 0x50
 8000752:	4b13      	ldr	r3, [pc, #76]	; (80007a0 <__sinit+0x68>)
 8000754:	4a13      	ldr	r2, [pc, #76]	; (80007a4 <__sinit+0x6c>)
 8000756:	681b      	ldr	r3, [r3, #0]
 8000758:	62a2      	str	r2, [r4, #40]	; 0x28
 800075a:	42a3      	cmp	r3, r4
 800075c:	bf04      	itt	eq
 800075e:	2301      	moveq	r3, #1
 8000760:	61a3      	streq	r3, [r4, #24]
 8000762:	4620      	mov	r0, r4
 8000764:	f000 f820 	bl	80007a8 <__sfp>
 8000768:	6060      	str	r0, [r4, #4]
 800076a:	4620      	mov	r0, r4
 800076c:	f000 f81c 	bl	80007a8 <__sfp>
 8000770:	60a0      	str	r0, [r4, #8]
 8000772:	4620      	mov	r0, r4
 8000774:	f000 f818 	bl	80007a8 <__sfp>
 8000778:	2200      	movs	r2, #0
 800077a:	60e0      	str	r0, [r4, #12]
 800077c:	2104      	movs	r1, #4
 800077e:	6860      	ldr	r0, [r4, #4]
 8000780:	f7ff ff82 	bl	8000688 <std>
 8000784:	68a0      	ldr	r0, [r4, #8]
 8000786:	2201      	movs	r2, #1
 8000788:	2109      	movs	r1, #9
 800078a:	f7ff ff7d 	bl	8000688 <std>
 800078e:	68e0      	ldr	r0, [r4, #12]
 8000790:	2202      	movs	r2, #2
 8000792:	2112      	movs	r1, #18
 8000794:	f7ff ff78 	bl	8000688 <std>
 8000798:	2301      	movs	r3, #1
 800079a:	61a3      	str	r3, [r4, #24]
 800079c:	e7d2      	b.n	8000744 <__sinit+0xc>
 800079e:	bf00      	nop
 80007a0:	08001534 	.word	0x08001534
 80007a4:	080006d1 	.word	0x080006d1

080007a8 <__sfp>:
 80007a8:	b5f8      	push	{r3, r4, r5, r6, r7, lr}
 80007aa:	4607      	mov	r7, r0
 80007ac:	f7ff ffac 	bl	8000708 <__sfp_lock_acquire>
 80007b0:	4b1e      	ldr	r3, [pc, #120]	; (800082c <__sfp+0x84>)
 80007b2:	681e      	ldr	r6, [r3, #0]
 80007b4:	69b3      	ldr	r3, [r6, #24]
 80007b6:	b913      	cbnz	r3, 80007be <__sfp+0x16>
 80007b8:	4630      	mov	r0, r6
 80007ba:	f7ff ffbd 	bl	8000738 <__sinit>
 80007be:	3648      	adds	r6, #72	; 0x48
 80007c0:	e9d6 3401 	ldrd	r3, r4, [r6, #4]
 80007c4:	3b01      	subs	r3, #1
 80007c6:	d503      	bpl.n	80007d0 <__sfp+0x28>
 80007c8:	6833      	ldr	r3, [r6, #0]
 80007ca:	b30b      	cbz	r3, 8000810 <__sfp+0x68>
 80007cc:	6836      	ldr	r6, [r6, #0]
 80007ce:	e7f7      	b.n	80007c0 <__sfp+0x18>
 80007d0:	f9b4 500c 	ldrsh.w	r5, [r4, #12]
 80007d4:	b9d5      	cbnz	r5, 800080c <__sfp+0x64>
 80007d6:	4b16      	ldr	r3, [pc, #88]	; (8000830 <__sfp+0x88>)
 80007d8:	60e3      	str	r3, [r4, #12]
 80007da:	f104 0058 	add.w	r0, r4, #88	; 0x58
 80007de:	6665      	str	r5, [r4, #100]	; 0x64
 80007e0:	f000 f847 	bl	8000872 <__retarget_lock_init_recursive>
 80007e4:	f7ff ff96 	bl	8000714 <__sfp_lock_release>
 80007e8:	e9c4 5501 	strd	r5, r5, [r4, #4]
 80007ec:	e9c4 5504 	strd	r5, r5, [r4, #16]
 80007f0:	6025      	str	r5, [r4, #0]
 80007f2:	61a5      	str	r5, [r4, #24]
 80007f4:	2208      	movs	r2, #8
 80007f6:	4629      	mov	r1, r5
 80007f8:	f104 005c 	add.w	r0, r4, #92	; 0x5c
 80007fc:	f7ff ff24 	bl	8000648 <memset>
 8000800:	e9c4 550d 	strd	r5, r5, [r4, #52]	; 0x34
 8000804:	e9c4 5512 	strd	r5, r5, [r4, #72]	; 0x48
 8000808:	4620      	mov	r0, r4
 800080a:	bdf8      	pop	{r3, r4, r5, r6, r7, pc}
 800080c:	3468      	adds	r4, #104	; 0x68
 800080e:	e7d9      	b.n	80007c4 <__sfp+0x1c>
 8000810:	2104      	movs	r1, #4
 8000812:	4638      	mov	r0, r7
 8000814:	f7ff ff62 	bl	80006dc <__sfmoreglue>
 8000818:	4604      	mov	r4, r0
 800081a:	6030      	str	r0, [r6, #0]
 800081c:	2800      	cmp	r0, #0
 800081e:	d1d5      	bne.n	80007cc <__sfp+0x24>
 8000820:	f7ff ff78 	bl	8000714 <__sfp_lock_release>
 8000824:	230c      	movs	r3, #12
 8000826:	603b      	str	r3, [r7, #0]
 8000828:	e7ee      	b.n	8000808 <__sfp+0x60>
 800082a:	bf00      	nop
 800082c:	08001534 	.word	0x08001534
 8000830:	ffff0001 	.word	0xffff0001

08000834 <_fwalk_reent>:
 8000834:	e92d 43f8 	stmdb	sp!, {r3, r4, r5, r6, r7, r8, r9, lr}
 8000838:	4606      	mov	r6, r0
 800083a:	4688      	mov	r8, r1
 800083c:	f100 0448 	add.w	r4, r0, #72	; 0x48
 8000840:	2700      	movs	r7, #0
 8000842:	e9d4 9501 	ldrd	r9, r5, [r4, #4]
 8000846:	f1b9 0901 	subs.w	r9, r9, #1
 800084a:	d505      	bpl.n	8000858 <_fwalk_reent+0x24>
 800084c:	6824      	ldr	r4, [r4, #0]
 800084e:	2c00      	cmp	r4, #0
 8000850:	d1f7      	bne.n	8000842 <_fwalk_reent+0xe>
 8000852:	4638      	mov	r0, r7
 8000854:	e8bd 83f8 	ldmia.w	sp!, {r3, r4, r5, r6, r7, r8, r9, pc}
 8000858:	89ab      	ldrh	r3, [r5, #12]
 800085a:	2b01      	cmp	r3, #1
 800085c:	d907      	bls.n	800086e <_fwalk_reent+0x3a>
 800085e:	f9b5 300e 	ldrsh.w	r3, [r5, #14]
 8000862:	3301      	adds	r3, #1
 8000864:	d003      	beq.n	800086e <_fwalk_reent+0x3a>
 8000866:	4629      	mov	r1, r5
 8000868:	4630      	mov	r0, r6
 800086a:	47c0      	blx	r8
 800086c:	4307      	orrs	r7, r0
 800086e:	3568      	adds	r5, #104	; 0x68
 8000870:	e7e9      	b.n	8000846 <_fwalk_reent+0x12>

08000872 <__retarget_lock_init_recursive>:
 8000872:	4770      	bx	lr

08000874 <__retarget_lock_acquire_recursive>:
 8000874:	4770      	bx	lr

08000876 <__retarget_lock_release_recursive>:
 8000876:	4770      	bx	lr

08000878 <_malloc_r>:
 8000878:	b5f8      	push	{r3, r4, r5, r6, r7, lr}
 800087a:	1ccd      	adds	r5, r1, #3
 800087c:	f025 0503 	bic.w	r5, r5, #3
 8000880:	3508      	adds	r5, #8
 8000882:	2d0c      	cmp	r5, #12
 8000884:	bf38      	it	cc
 8000886:	250c      	movcc	r5, #12
 8000888:	2d00      	cmp	r5, #0
 800088a:	4606      	mov	r6, r0
 800088c:	db01      	blt.n	8000892 <_malloc_r+0x1a>
 800088e:	42a9      	cmp	r1, r5
 8000890:	d903      	bls.n	800089a <_malloc_r+0x22>
 8000892:	230c      	movs	r3, #12
 8000894:	6033      	str	r3, [r6, #0]
 8000896:	2000      	movs	r0, #0
 8000898:	bdf8      	pop	{r3, r4, r5, r6, r7, pc}
 800089a:	f000 fda3 	bl	80013e4 <__malloc_lock>
 800089e:	4921      	ldr	r1, [pc, #132]	; (8000924 <_malloc_r+0xac>)
 80008a0:	680a      	ldr	r2, [r1, #0]
 80008a2:	4614      	mov	r4, r2
 80008a4:	b99c      	cbnz	r4, 80008ce <_malloc_r+0x56>
 80008a6:	4f20      	ldr	r7, [pc, #128]	; (8000928 <_malloc_r+0xb0>)
 80008a8:	683b      	ldr	r3, [r7, #0]
 80008aa:	b923      	cbnz	r3, 80008b6 <_malloc_r+0x3e>
 80008ac:	4621      	mov	r1, r4
 80008ae:	4630      	mov	r0, r6
 80008b0:	f000 fb2a 	bl	8000f08 <_sbrk_r>
 80008b4:	6038      	str	r0, [r7, #0]
 80008b6:	4629      	mov	r1, r5
 80008b8:	4630      	mov	r0, r6
 80008ba:	f000 fb25 	bl	8000f08 <_sbrk_r>
 80008be:	1c43      	adds	r3, r0, #1
 80008c0:	d123      	bne.n	800090a <_malloc_r+0x92>
 80008c2:	230c      	movs	r3, #12
 80008c4:	6033      	str	r3, [r6, #0]
 80008c6:	4630      	mov	r0, r6
 80008c8:	f000 fd92 	bl	80013f0 <__malloc_unlock>
 80008cc:	e7e3      	b.n	8000896 <_malloc_r+0x1e>
 80008ce:	6823      	ldr	r3, [r4, #0]
 80008d0:	1b5b      	subs	r3, r3, r5
 80008d2:	d417      	bmi.n	8000904 <_malloc_r+0x8c>
 80008d4:	2b0b      	cmp	r3, #11
 80008d6:	d903      	bls.n	80008e0 <_malloc_r+0x68>
 80008d8:	6023      	str	r3, [r4, #0]
 80008da:	441c      	add	r4, r3
 80008dc:	6025      	str	r5, [r4, #0]
 80008de:	e004      	b.n	80008ea <_malloc_r+0x72>
 80008e0:	6863      	ldr	r3, [r4, #4]
 80008e2:	42a2      	cmp	r2, r4
 80008e4:	bf0c      	ite	eq
 80008e6:	600b      	streq	r3, [r1, #0]
 80008e8:	6053      	strne	r3, [r2, #4]
 80008ea:	4630      	mov	r0, r6
 80008ec:	f000 fd80 	bl	80013f0 <__malloc_unlock>
 80008f0:	f104 000b 	add.w	r0, r4, #11
 80008f4:	1d23      	adds	r3, r4, #4
 80008f6:	f020 0007 	bic.w	r0, r0, #7
 80008fa:	1ac2      	subs	r2, r0, r3
 80008fc:	d0cc      	beq.n	8000898 <_malloc_r+0x20>
 80008fe:	1a1b      	subs	r3, r3, r0
 8000900:	50a3      	str	r3, [r4, r2]
 8000902:	e7c9      	b.n	8000898 <_malloc_r+0x20>
 8000904:	4622      	mov	r2, r4
 8000906:	6864      	ldr	r4, [r4, #4]
 8000908:	e7cc      	b.n	80008a4 <_malloc_r+0x2c>
 800090a:	1cc4      	adds	r4, r0, #3
 800090c:	f024 0403 	bic.w	r4, r4, #3
 8000910:	42a0      	cmp	r0, r4
 8000912:	d0e3      	beq.n	80008dc <_malloc_r+0x64>
 8000914:	1a21      	subs	r1, r4, r0
 8000916:	4630      	mov	r0, r6
 8000918:	f000 faf6 	bl	8000f08 <_sbrk_r>
 800091c:	3001      	adds	r0, #1
 800091e:	d1dd      	bne.n	80008dc <_malloc_r+0x64>
 8000920:	e7cf      	b.n	80008c2 <_malloc_r+0x4a>
 8000922:	bf00      	nop
 8000924:	20000084 	.word	0x20000084
 8000928:	20000088 	.word	0x20000088

0800092c <__sfputc_r>:
 800092c:	6893      	ldr	r3, [r2, #8]
 800092e:	3b01      	subs	r3, #1
 8000930:	2b00      	cmp	r3, #0
 8000932:	b410      	push	{r4}
 8000934:	6093      	str	r3, [r2, #8]
 8000936:	da08      	bge.n	800094a <__sfputc_r+0x1e>
 8000938:	6994      	ldr	r4, [r2, #24]
 800093a:	42a3      	cmp	r3, r4
 800093c:	db01      	blt.n	8000942 <__sfputc_r+0x16>
 800093e:	290a      	cmp	r1, #10
 8000940:	d103      	bne.n	800094a <__sfputc_r+0x1e>
 8000942:	f85d 4b04 	ldr.w	r4, [sp], #4
 8000946:	f000 bb33 	b.w	8000fb0 <__swbuf_r>
 800094a:	6813      	ldr	r3, [r2, #0]
 800094c:	1c58      	adds	r0, r3, #1
 800094e:	6010      	str	r0, [r2, #0]
 8000950:	7019      	strb	r1, [r3, #0]
 8000952:	4608      	mov	r0, r1
 8000954:	f85d 4b04 	ldr.w	r4, [sp], #4
 8000958:	4770      	bx	lr

0800095a <__sfputs_r>:
 800095a:	b5f8      	push	{r3, r4, r5, r6, r7, lr}
 800095c:	4606      	mov	r6, r0
 800095e:	460f      	mov	r7, r1
 8000960:	4614      	mov	r4, r2
 8000962:	18d5      	adds	r5, r2, r3
 8000964:	42ac      	cmp	r4, r5
 8000966:	d101      	bne.n	800096c <__sfputs_r+0x12>
 8000968:	2000      	movs	r0, #0
 800096a:	e007      	b.n	800097c <__sfputs_r+0x22>
 800096c:	f814 1b01 	ldrb.w	r1, [r4], #1
 8000970:	463a      	mov	r2, r7
 8000972:	4630      	mov	r0, r6
 8000974:	f7ff ffda 	bl	800092c <__sfputc_r>
 8000978:	1c43      	adds	r3, r0, #1
 800097a:	d1f3      	bne.n	8000964 <__sfputs_r+0xa>
 800097c:	bdf8      	pop	{r3, r4, r5, r6, r7, pc}
	...

08000980 <_vfiprintf_r>:
 8000980:	e92d 4ff0 	stmdb	sp!, {r4, r5, r6, r7, r8, r9, sl, fp, lr}
 8000984:	460d      	mov	r5, r1
 8000986:	b09d      	sub	sp, #116	; 0x74
 8000988:	4614      	mov	r4, r2
 800098a:	4698      	mov	r8, r3
 800098c:	4606      	mov	r6, r0
 800098e:	b118      	cbz	r0, 8000998 <_vfiprintf_r+0x18>
 8000990:	6983      	ldr	r3, [r0, #24]
 8000992:	b90b      	cbnz	r3, 8000998 <_vfiprintf_r+0x18>
 8000994:	f7ff fed0 	bl	8000738 <__sinit>
 8000998:	4b89      	ldr	r3, [pc, #548]	; (8000bc0 <_vfiprintf_r+0x240>)
 800099a:	429d      	cmp	r5, r3
 800099c:	d11b      	bne.n	80009d6 <_vfiprintf_r+0x56>
 800099e:	6875      	ldr	r5, [r6, #4]
 80009a0:	6e6b      	ldr	r3, [r5, #100]	; 0x64
 80009a2:	07d9      	lsls	r1, r3, #31
 80009a4:	d405      	bmi.n	80009b2 <_vfiprintf_r+0x32>
 80009a6:	89ab      	ldrh	r3, [r5, #12]
 80009a8:	059a      	lsls	r2, r3, #22
 80009aa:	d402      	bmi.n	80009b2 <_vfiprintf_r+0x32>
 80009ac:	6da8      	ldr	r0, [r5, #88]	; 0x58
 80009ae:	f7ff ff61 	bl	8000874 <__retarget_lock_acquire_recursive>
 80009b2:	89ab      	ldrh	r3, [r5, #12]
 80009b4:	071b      	lsls	r3, r3, #28
 80009b6:	d501      	bpl.n	80009bc <_vfiprintf_r+0x3c>
 80009b8:	692b      	ldr	r3, [r5, #16]
 80009ba:	b9eb      	cbnz	r3, 80009f8 <_vfiprintf_r+0x78>
 80009bc:	4629      	mov	r1, r5
 80009be:	4630      	mov	r0, r6
 80009c0:	f000 fb5a 	bl	8001078 <__swsetup_r>
 80009c4:	b1c0      	cbz	r0, 80009f8 <_vfiprintf_r+0x78>
 80009c6:	6e6b      	ldr	r3, [r5, #100]	; 0x64
 80009c8:	07dc      	lsls	r4, r3, #31
 80009ca:	d50e      	bpl.n	80009ea <_vfiprintf_r+0x6a>
 80009cc:	f04f 30ff 	mov.w	r0, #4294967295
 80009d0:	b01d      	add	sp, #116	; 0x74
 80009d2:	e8bd 8ff0 	ldmia.w	sp!, {r4, r5, r6, r7, r8, r9, sl, fp, pc}
 80009d6:	4b7b      	ldr	r3, [pc, #492]	; (8000bc4 <_vfiprintf_r+0x244>)
 80009d8:	429d      	cmp	r5, r3
 80009da:	d101      	bne.n	80009e0 <_vfiprintf_r+0x60>
 80009dc:	68b5      	ldr	r5, [r6, #8]
 80009de:	e7df      	b.n	80009a0 <_vfiprintf_r+0x20>
 80009e0:	4b79      	ldr	r3, [pc, #484]	; (8000bc8 <_vfiprintf_r+0x248>)
 80009e2:	429d      	cmp	r5, r3
 80009e4:	bf08      	it	eq
 80009e6:	68f5      	ldreq	r5, [r6, #12]
 80009e8:	e7da      	b.n	80009a0 <_vfiprintf_r+0x20>
 80009ea:	89ab      	ldrh	r3, [r5, #12]
 80009ec:	0598      	lsls	r0, r3, #22
 80009ee:	d4ed      	bmi.n	80009cc <_vfiprintf_r+0x4c>
 80009f0:	6da8      	ldr	r0, [r5, #88]	; 0x58
 80009f2:	f7ff ff40 	bl	8000876 <__retarget_lock_release_recursive>
 80009f6:	e7e9      	b.n	80009cc <_vfiprintf_r+0x4c>
 80009f8:	2300      	movs	r3, #0
 80009fa:	9309      	str	r3, [sp, #36]	; 0x24
 80009fc:	2320      	movs	r3, #32
 80009fe:	f88d 3029 	strb.w	r3, [sp, #41]	; 0x29
 8000a02:	f8cd 800c 	str.w	r8, [sp, #12]
 8000a06:	2330      	movs	r3, #48	; 0x30
 8000a08:	f8df 81c0 	ldr.w	r8, [pc, #448]	; 8000bcc <_vfiprintf_r+0x24c>
 8000a0c:	f88d 302a 	strb.w	r3, [sp, #42]	; 0x2a
 8000a10:	f04f 0901 	mov.w	r9, #1
 8000a14:	4623      	mov	r3, r4
 8000a16:	469a      	mov	sl, r3
 8000a18:	f813 2b01 	ldrb.w	r2, [r3], #1
 8000a1c:	b10a      	cbz	r2, 8000a22 <_vfiprintf_r+0xa2>
 8000a1e:	2a25      	cmp	r2, #37	; 0x25
 8000a20:	d1f9      	bne.n	8000a16 <_vfiprintf_r+0x96>
 8000a22:	ebba 0b04 	subs.w	fp, sl, r4
 8000a26:	d00b      	beq.n	8000a40 <_vfiprintf_r+0xc0>
 8000a28:	465b      	mov	r3, fp
 8000a2a:	4622      	mov	r2, r4
 8000a2c:	4629      	mov	r1, r5
 8000a2e:	4630      	mov	r0, r6
 8000a30:	f7ff ff93 	bl	800095a <__sfputs_r>
 8000a34:	3001      	adds	r0, #1
 8000a36:	f000 80aa 	beq.w	8000b8e <_vfiprintf_r+0x20e>
 8000a3a:	9a09      	ldr	r2, [sp, #36]	; 0x24
 8000a3c:	445a      	add	r2, fp
 8000a3e:	9209      	str	r2, [sp, #36]	; 0x24
 8000a40:	f89a 3000 	ldrb.w	r3, [sl]
 8000a44:	2b00      	cmp	r3, #0
 8000a46:	f000 80a2 	beq.w	8000b8e <_vfiprintf_r+0x20e>
 8000a4a:	2300      	movs	r3, #0
 8000a4c:	f04f 32ff 	mov.w	r2, #4294967295
 8000a50:	e9cd 2305 	strd	r2, r3, [sp, #20]
 8000a54:	f10a 0a01 	add.w	sl, sl, #1
 8000a58:	9304      	str	r3, [sp, #16]
 8000a5a:	9307      	str	r3, [sp, #28]
 8000a5c:	f88d 3053 	strb.w	r3, [sp, #83]	; 0x53
 8000a60:	931a      	str	r3, [sp, #104]	; 0x68
 8000a62:	4654      	mov	r4, sl
 8000a64:	2205      	movs	r2, #5
 8000a66:	f814 1b01 	ldrb.w	r1, [r4], #1
 8000a6a:	4858      	ldr	r0, [pc, #352]	; (8000bcc <_vfiprintf_r+0x24c>)
 8000a6c:	f7ff fbb8 	bl	80001e0 <memchr>
 8000a70:	9a04      	ldr	r2, [sp, #16]
 8000a72:	b9d8      	cbnz	r0, 8000aac <_vfiprintf_r+0x12c>
 8000a74:	06d1      	lsls	r1, r2, #27
 8000a76:	bf44      	itt	mi
 8000a78:	2320      	movmi	r3, #32
 8000a7a:	f88d 3053 	strbmi.w	r3, [sp, #83]	; 0x53
 8000a7e:	0713      	lsls	r3, r2, #28
 8000a80:	bf44      	itt	mi
 8000a82:	232b      	movmi	r3, #43	; 0x2b
 8000a84:	f88d 3053 	strbmi.w	r3, [sp, #83]	; 0x53
 8000a88:	f89a 3000 	ldrb.w	r3, [sl]
 8000a8c:	2b2a      	cmp	r3, #42	; 0x2a
 8000a8e:	d015      	beq.n	8000abc <_vfiprintf_r+0x13c>
 8000a90:	9a07      	ldr	r2, [sp, #28]
 8000a92:	4654      	mov	r4, sl
 8000a94:	2000      	movs	r0, #0
 8000a96:	f04f 0c0a 	mov.w	ip, #10
 8000a9a:	4621      	mov	r1, r4
 8000a9c:	f811 3b01 	ldrb.w	r3, [r1], #1
 8000aa0:	3b30      	subs	r3, #48	; 0x30
 8000aa2:	2b09      	cmp	r3, #9
 8000aa4:	d94e      	bls.n	8000b44 <_vfiprintf_r+0x1c4>
 8000aa6:	b1b0      	cbz	r0, 8000ad6 <_vfiprintf_r+0x156>
 8000aa8:	9207      	str	r2, [sp, #28]
 8000aaa:	e014      	b.n	8000ad6 <_vfiprintf_r+0x156>
 8000aac:	eba0 0308 	sub.w	r3, r0, r8
 8000ab0:	fa09 f303 	lsl.w	r3, r9, r3
 8000ab4:	4313      	orrs	r3, r2
 8000ab6:	9304      	str	r3, [sp, #16]
 8000ab8:	46a2      	mov	sl, r4
 8000aba:	e7d2      	b.n	8000a62 <_vfiprintf_r+0xe2>
 8000abc:	9b03      	ldr	r3, [sp, #12]
 8000abe:	1d19      	adds	r1, r3, #4
 8000ac0:	681b      	ldr	r3, [r3, #0]
 8000ac2:	9103      	str	r1, [sp, #12]
 8000ac4:	2b00      	cmp	r3, #0
 8000ac6:	bfbb      	ittet	lt
 8000ac8:	425b      	neglt	r3, r3
 8000aca:	f042 0202 	orrlt.w	r2, r2, #2
 8000ace:	9307      	strge	r3, [sp, #28]
 8000ad0:	9307      	strlt	r3, [sp, #28]
 8000ad2:	bfb8      	it	lt
 8000ad4:	9204      	strlt	r2, [sp, #16]
 8000ad6:	7823      	ldrb	r3, [r4, #0]
 8000ad8:	2b2e      	cmp	r3, #46	; 0x2e
 8000ada:	d10c      	bne.n	8000af6 <_vfiprintf_r+0x176>
 8000adc:	7863      	ldrb	r3, [r4, #1]
 8000ade:	2b2a      	cmp	r3, #42	; 0x2a
 8000ae0:	d135      	bne.n	8000b4e <_vfiprintf_r+0x1ce>
 8000ae2:	9b03      	ldr	r3, [sp, #12]
 8000ae4:	1d1a      	adds	r2, r3, #4
 8000ae6:	681b      	ldr	r3, [r3, #0]
 8000ae8:	9203      	str	r2, [sp, #12]
 8000aea:	2b00      	cmp	r3, #0
 8000aec:	bfb8      	it	lt
 8000aee:	f04f 33ff 	movlt.w	r3, #4294967295
 8000af2:	3402      	adds	r4, #2
 8000af4:	9305      	str	r3, [sp, #20]
 8000af6:	f8df a0e4 	ldr.w	sl, [pc, #228]	; 8000bdc <_vfiprintf_r+0x25c>
 8000afa:	7821      	ldrb	r1, [r4, #0]
 8000afc:	2203      	movs	r2, #3
 8000afe:	4650      	mov	r0, sl
 8000b00:	f7ff fb6e 	bl	80001e0 <memchr>
 8000b04:	b140      	cbz	r0, 8000b18 <_vfiprintf_r+0x198>
 8000b06:	2340      	movs	r3, #64	; 0x40
 8000b08:	eba0 000a 	sub.w	r0, r0, sl
 8000b0c:	fa03 f000 	lsl.w	r0, r3, r0
 8000b10:	9b04      	ldr	r3, [sp, #16]
 8000b12:	4303      	orrs	r3, r0
 8000b14:	3401      	adds	r4, #1
 8000b16:	9304      	str	r3, [sp, #16]
 8000b18:	f814 1b01 	ldrb.w	r1, [r4], #1
 8000b1c:	482c      	ldr	r0, [pc, #176]	; (8000bd0 <_vfiprintf_r+0x250>)
 8000b1e:	f88d 1028 	strb.w	r1, [sp, #40]	; 0x28
 8000b22:	2206      	movs	r2, #6
 8000b24:	f7ff fb5c 	bl	80001e0 <memchr>
 8000b28:	2800      	cmp	r0, #0
 8000b2a:	d03f      	beq.n	8000bac <_vfiprintf_r+0x22c>
 8000b2c:	4b29      	ldr	r3, [pc, #164]	; (8000bd4 <_vfiprintf_r+0x254>)
 8000b2e:	bb1b      	cbnz	r3, 8000b78 <_vfiprintf_r+0x1f8>
 8000b30:	9b03      	ldr	r3, [sp, #12]
 8000b32:	3307      	adds	r3, #7
 8000b34:	f023 0307 	bic.w	r3, r3, #7
 8000b38:	3308      	adds	r3, #8
 8000b3a:	9303      	str	r3, [sp, #12]
 8000b3c:	9b09      	ldr	r3, [sp, #36]	; 0x24
 8000b3e:	443b      	add	r3, r7
 8000b40:	9309      	str	r3, [sp, #36]	; 0x24
 8000b42:	e767      	b.n	8000a14 <_vfiprintf_r+0x94>
 8000b44:	fb0c 3202 	mla	r2, ip, r2, r3
 8000b48:	460c      	mov	r4, r1
 8000b4a:	2001      	movs	r0, #1
 8000b4c:	e7a5      	b.n	8000a9a <_vfiprintf_r+0x11a>
 8000b4e:	2300      	movs	r3, #0
 8000b50:	3401      	adds	r4, #1
 8000b52:	9305      	str	r3, [sp, #20]
 8000b54:	4619      	mov	r1, r3
 8000b56:	f04f 0c0a 	mov.w	ip, #10
 8000b5a:	4620      	mov	r0, r4
 8000b5c:	f810 2b01 	ldrb.w	r2, [r0], #1
 8000b60:	3a30      	subs	r2, #48	; 0x30
 8000b62:	2a09      	cmp	r2, #9
 8000b64:	d903      	bls.n	8000b6e <_vfiprintf_r+0x1ee>
 8000b66:	2b00      	cmp	r3, #0
 8000b68:	d0c5      	beq.n	8000af6 <_vfiprintf_r+0x176>
 8000b6a:	9105      	str	r1, [sp, #20]
 8000b6c:	e7c3      	b.n	8000af6 <_vfiprintf_r+0x176>
 8000b6e:	fb0c 2101 	mla	r1, ip, r1, r2
 8000b72:	4604      	mov	r4, r0
 8000b74:	2301      	movs	r3, #1
 8000b76:	e7f0      	b.n	8000b5a <_vfiprintf_r+0x1da>
 8000b78:	ab03      	add	r3, sp, #12
 8000b7a:	9300      	str	r3, [sp, #0]
 8000b7c:	462a      	mov	r2, r5
 8000b7e:	4b16      	ldr	r3, [pc, #88]	; (8000bd8 <_vfiprintf_r+0x258>)
 8000b80:	a904      	add	r1, sp, #16
 8000b82:	4630      	mov	r0, r6
 8000b84:	f3af 8000 	nop.w
 8000b88:	4607      	mov	r7, r0
 8000b8a:	1c78      	adds	r0, r7, #1
 8000b8c:	d1d6      	bne.n	8000b3c <_vfiprintf_r+0x1bc>
 8000b8e:	6e6b      	ldr	r3, [r5, #100]	; 0x64
 8000b90:	07d9      	lsls	r1, r3, #31
 8000b92:	d405      	bmi.n	8000ba0 <_vfiprintf_r+0x220>
 8000b94:	89ab      	ldrh	r3, [r5, #12]
 8000b96:	059a      	lsls	r2, r3, #22
 8000b98:	d402      	bmi.n	8000ba0 <_vfiprintf_r+0x220>
 8000b9a:	6da8      	ldr	r0, [r5, #88]	; 0x58
 8000b9c:	f7ff fe6b 	bl	8000876 <__retarget_lock_release_recursive>
 8000ba0:	89ab      	ldrh	r3, [r5, #12]
 8000ba2:	065b      	lsls	r3, r3, #25
 8000ba4:	f53f af12 	bmi.w	80009cc <_vfiprintf_r+0x4c>
 8000ba8:	9809      	ldr	r0, [sp, #36]	; 0x24
 8000baa:	e711      	b.n	80009d0 <_vfiprintf_r+0x50>
 8000bac:	ab03      	add	r3, sp, #12
 8000bae:	9300      	str	r3, [sp, #0]
 8000bb0:	462a      	mov	r2, r5
 8000bb2:	4b09      	ldr	r3, [pc, #36]	; (8000bd8 <_vfiprintf_r+0x258>)
 8000bb4:	a904      	add	r1, sp, #16
 8000bb6:	4630      	mov	r0, r6
 8000bb8:	f000 f880 	bl	8000cbc <_printf_i>
 8000bbc:	e7e4      	b.n	8000b88 <_vfiprintf_r+0x208>
 8000bbe:	bf00      	nop
 8000bc0:	08001558 	.word	0x08001558
 8000bc4:	08001578 	.word	0x08001578
 8000bc8:	08001538 	.word	0x08001538
 8000bcc:	08001598 	.word	0x08001598
 8000bd0:	080015a2 	.word	0x080015a2
 8000bd4:	00000000 	.word	0x00000000
 8000bd8:	0800095b 	.word	0x0800095b
 8000bdc:	0800159e 	.word	0x0800159e

08000be0 <_printf_common>:
 8000be0:	e92d 47f0 	stmdb	sp!, {r4, r5, r6, r7, r8, r9, sl, lr}
 8000be4:	4616      	mov	r6, r2
 8000be6:	4699      	mov	r9, r3
 8000be8:	688a      	ldr	r2, [r1, #8]
 8000bea:	690b      	ldr	r3, [r1, #16]
 8000bec:	f8dd 8020 	ldr.w	r8, [sp, #32]
 8000bf0:	4293      	cmp	r3, r2
 8000bf2:	bfb8      	it	lt
 8000bf4:	4613      	movlt	r3, r2
 8000bf6:	6033      	str	r3, [r6, #0]
 8000bf8:	f891 2043 	ldrb.w	r2, [r1, #67]	; 0x43
 8000bfc:	4607      	mov	r7, r0
 8000bfe:	460c      	mov	r4, r1
 8000c00:	b10a      	cbz	r2, 8000c06 <_printf_common+0x26>
 8000c02:	3301      	adds	r3, #1
 8000c04:	6033      	str	r3, [r6, #0]
 8000c06:	6823      	ldr	r3, [r4, #0]
 8000c08:	0699      	lsls	r1, r3, #26
 8000c0a:	bf42      	ittt	mi
 8000c0c:	6833      	ldrmi	r3, [r6, #0]
 8000c0e:	3302      	addmi	r3, #2
 8000c10:	6033      	strmi	r3, [r6, #0]
 8000c12:	6825      	ldr	r5, [r4, #0]
 8000c14:	f015 0506 	ands.w	r5, r5, #6
 8000c18:	d106      	bne.n	8000c28 <_printf_common+0x48>
 8000c1a:	f104 0a19 	add.w	sl, r4, #25
 8000c1e:	68e3      	ldr	r3, [r4, #12]
 8000c20:	6832      	ldr	r2, [r6, #0]
 8000c22:	1a9b      	subs	r3, r3, r2
 8000c24:	42ab      	cmp	r3, r5
 8000c26:	dc26      	bgt.n	8000c76 <_printf_common+0x96>
 8000c28:	f894 2043 	ldrb.w	r2, [r4, #67]	; 0x43
 8000c2c:	1e13      	subs	r3, r2, #0
 8000c2e:	6822      	ldr	r2, [r4, #0]
 8000c30:	bf18      	it	ne
 8000c32:	2301      	movne	r3, #1
 8000c34:	0692      	lsls	r2, r2, #26
 8000c36:	d42b      	bmi.n	8000c90 <_printf_common+0xb0>
 8000c38:	f104 0243 	add.w	r2, r4, #67	; 0x43
 8000c3c:	4649      	mov	r1, r9
 8000c3e:	4638      	mov	r0, r7
 8000c40:	47c0      	blx	r8
 8000c42:	3001      	adds	r0, #1
 8000c44:	d01e      	beq.n	8000c84 <_printf_common+0xa4>
 8000c46:	6823      	ldr	r3, [r4, #0]
 8000c48:	68e5      	ldr	r5, [r4, #12]
 8000c4a:	6832      	ldr	r2, [r6, #0]
 8000c4c:	f003 0306 	and.w	r3, r3, #6
 8000c50:	2b04      	cmp	r3, #4
 8000c52:	bf08      	it	eq
 8000c54:	1aad      	subeq	r5, r5, r2
 8000c56:	68a3      	ldr	r3, [r4, #8]
 8000c58:	6922      	ldr	r2, [r4, #16]
 8000c5a:	bf0c      	ite	eq
 8000c5c:	ea25 75e5 	biceq.w	r5, r5, r5, asr #31
 8000c60:	2500      	movne	r5, #0
 8000c62:	4293      	cmp	r3, r2
 8000c64:	bfc4      	itt	gt
 8000c66:	1a9b      	subgt	r3, r3, r2
 8000c68:	18ed      	addgt	r5, r5, r3
 8000c6a:	2600      	movs	r6, #0
 8000c6c:	341a      	adds	r4, #26
 8000c6e:	42b5      	cmp	r5, r6
 8000c70:	d11a      	bne.n	8000ca8 <_printf_common+0xc8>
 8000c72:	2000      	movs	r0, #0
 8000c74:	e008      	b.n	8000c88 <_printf_common+0xa8>
 8000c76:	2301      	movs	r3, #1
 8000c78:	4652      	mov	r2, sl
 8000c7a:	4649      	mov	r1, r9
 8000c7c:	4638      	mov	r0, r7
 8000c7e:	47c0      	blx	r8
 8000c80:	3001      	adds	r0, #1
 8000c82:	d103      	bne.n	8000c8c <_printf_common+0xac>
 8000c84:	f04f 30ff 	mov.w	r0, #4294967295
 8000c88:	e8bd 87f0 	ldmia.w	sp!, {r4, r5, r6, r7, r8, r9, sl, pc}
 8000c8c:	3501      	adds	r5, #1
 8000c8e:	e7c6      	b.n	8000c1e <_printf_common+0x3e>
 8000c90:	18e1      	adds	r1, r4, r3
 8000c92:	1c5a      	adds	r2, r3, #1
 8000c94:	2030      	movs	r0, #48	; 0x30
 8000c96:	f881 0043 	strb.w	r0, [r1, #67]	; 0x43
 8000c9a:	4422      	add	r2, r4
 8000c9c:	f894 1045 	ldrb.w	r1, [r4, #69]	; 0x45
 8000ca0:	f882 1043 	strb.w	r1, [r2, #67]	; 0x43
 8000ca4:	3302      	adds	r3, #2
 8000ca6:	e7c7      	b.n	8000c38 <_printf_common+0x58>
 8000ca8:	2301      	movs	r3, #1
 8000caa:	4622      	mov	r2, r4
 8000cac:	4649      	mov	r1, r9
 8000cae:	4638      	mov	r0, r7
 8000cb0:	47c0      	blx	r8
 8000cb2:	3001      	adds	r0, #1
 8000cb4:	d0e6      	beq.n	8000c84 <_printf_common+0xa4>
 8000cb6:	3601      	adds	r6, #1
 8000cb8:	e7d9      	b.n	8000c6e <_printf_common+0x8e>
	...

08000cbc <_printf_i>:
 8000cbc:	e92d 47ff 	stmdb	sp!, {r0, r1, r2, r3, r4, r5, r6, r7, r8, r9, sl, lr}
 8000cc0:	460c      	mov	r4, r1
 8000cc2:	4691      	mov	r9, r2
 8000cc4:	7e27      	ldrb	r7, [r4, #24]
 8000cc6:	990c      	ldr	r1, [sp, #48]	; 0x30
 8000cc8:	2f78      	cmp	r7, #120	; 0x78
 8000cca:	4680      	mov	r8, r0
 8000ccc:	469a      	mov	sl, r3
 8000cce:	f104 0243 	add.w	r2, r4, #67	; 0x43
 8000cd2:	d807      	bhi.n	8000ce4 <_printf_i+0x28>
 8000cd4:	2f62      	cmp	r7, #98	; 0x62
 8000cd6:	d80a      	bhi.n	8000cee <_printf_i+0x32>
 8000cd8:	2f00      	cmp	r7, #0
 8000cda:	f000 80d8 	beq.w	8000e8e <_printf_i+0x1d2>
 8000cde:	2f58      	cmp	r7, #88	; 0x58
 8000ce0:	f000 80a3 	beq.w	8000e2a <_printf_i+0x16e>
 8000ce4:	f104 0642 	add.w	r6, r4, #66	; 0x42
 8000ce8:	f884 7042 	strb.w	r7, [r4, #66]	; 0x42
 8000cec:	e03a      	b.n	8000d64 <_printf_i+0xa8>
 8000cee:	f1a7 0363 	sub.w	r3, r7, #99	; 0x63
 8000cf2:	2b15      	cmp	r3, #21
 8000cf4:	d8f6      	bhi.n	8000ce4 <_printf_i+0x28>
 8000cf6:	a001      	add	r0, pc, #4	; (adr r0, 8000cfc <_printf_i+0x40>)
 8000cf8:	f850 f023 	ldr.w	pc, [r0, r3, lsl #2]
 8000cfc:	08000d55 	.word	0x08000d55
 8000d00:	08000d69 	.word	0x08000d69
 8000d04:	08000ce5 	.word	0x08000ce5
 8000d08:	08000ce5 	.word	0x08000ce5
 8000d0c:	08000ce5 	.word	0x08000ce5
 8000d10:	08000ce5 	.word	0x08000ce5
 8000d14:	08000d69 	.word	0x08000d69
 8000d18:	08000ce5 	.word	0x08000ce5
 8000d1c:	08000ce5 	.word	0x08000ce5
 8000d20:	08000ce5 	.word	0x08000ce5
 8000d24:	08000ce5 	.word	0x08000ce5
 8000d28:	08000e75 	.word	0x08000e75
 8000d2c:	08000d99 	.word	0x08000d99
 8000d30:	08000e57 	.word	0x08000e57
 8000d34:	08000ce5 	.word	0x08000ce5
 8000d38:	08000ce5 	.word	0x08000ce5
 8000d3c:	08000e97 	.word	0x08000e97
 8000d40:	08000ce5 	.word	0x08000ce5
 8000d44:	08000d99 	.word	0x08000d99
 8000d48:	08000ce5 	.word	0x08000ce5
 8000d4c:	08000ce5 	.word	0x08000ce5
 8000d50:	08000e5f 	.word	0x08000e5f
 8000d54:	680b      	ldr	r3, [r1, #0]
 8000d56:	1d1a      	adds	r2, r3, #4
 8000d58:	681b      	ldr	r3, [r3, #0]
 8000d5a:	600a      	str	r2, [r1, #0]
 8000d5c:	f104 0642 	add.w	r6, r4, #66	; 0x42
 8000d60:	f884 3042 	strb.w	r3, [r4, #66]	; 0x42
 8000d64:	2301      	movs	r3, #1
 8000d66:	e0a3      	b.n	8000eb0 <_printf_i+0x1f4>
 8000d68:	6825      	ldr	r5, [r4, #0]
 8000d6a:	6808      	ldr	r0, [r1, #0]
 8000d6c:	062e      	lsls	r6, r5, #24
 8000d6e:	f100 0304 	add.w	r3, r0, #4
 8000d72:	d50a      	bpl.n	8000d8a <_printf_i+0xce>
 8000d74:	6805      	ldr	r5, [r0, #0]
 8000d76:	600b      	str	r3, [r1, #0]
 8000d78:	2d00      	cmp	r5, #0
 8000d7a:	da03      	bge.n	8000d84 <_printf_i+0xc8>
 8000d7c:	232d      	movs	r3, #45	; 0x2d
 8000d7e:	426d      	negs	r5, r5
 8000d80:	f884 3043 	strb.w	r3, [r4, #67]	; 0x43
 8000d84:	485e      	ldr	r0, [pc, #376]	; (8000f00 <_printf_i+0x244>)
 8000d86:	230a      	movs	r3, #10
 8000d88:	e019      	b.n	8000dbe <_printf_i+0x102>
 8000d8a:	f015 0f40 	tst.w	r5, #64	; 0x40
 8000d8e:	6805      	ldr	r5, [r0, #0]
 8000d90:	600b      	str	r3, [r1, #0]
 8000d92:	bf18      	it	ne
 8000d94:	b22d      	sxthne	r5, r5
 8000d96:	e7ef      	b.n	8000d78 <_printf_i+0xbc>
 8000d98:	680b      	ldr	r3, [r1, #0]
 8000d9a:	6825      	ldr	r5, [r4, #0]
 8000d9c:	1d18      	adds	r0, r3, #4
 8000d9e:	6008      	str	r0, [r1, #0]
 8000da0:	0628      	lsls	r0, r5, #24
 8000da2:	d501      	bpl.n	8000da8 <_printf_i+0xec>
 8000da4:	681d      	ldr	r5, [r3, #0]
 8000da6:	e002      	b.n	8000dae <_printf_i+0xf2>
 8000da8:	0669      	lsls	r1, r5, #25
 8000daa:	d5fb      	bpl.n	8000da4 <_printf_i+0xe8>
 8000dac:	881d      	ldrh	r5, [r3, #0]
 8000dae:	4854      	ldr	r0, [pc, #336]	; (8000f00 <_printf_i+0x244>)
 8000db0:	2f6f      	cmp	r7, #111	; 0x6f
 8000db2:	bf0c      	ite	eq
 8000db4:	2308      	moveq	r3, #8
 8000db6:	230a      	movne	r3, #10
 8000db8:	2100      	movs	r1, #0
 8000dba:	f884 1043 	strb.w	r1, [r4, #67]	; 0x43
 8000dbe:	6866      	ldr	r6, [r4, #4]
 8000dc0:	60a6      	str	r6, [r4, #8]
 8000dc2:	2e00      	cmp	r6, #0
 8000dc4:	bfa2      	ittt	ge
 8000dc6:	6821      	ldrge	r1, [r4, #0]
 8000dc8:	f021 0104 	bicge.w	r1, r1, #4
 8000dcc:	6021      	strge	r1, [r4, #0]
 8000dce:	b90d      	cbnz	r5, 8000dd4 <_printf_i+0x118>
 8000dd0:	2e00      	cmp	r6, #0
 8000dd2:	d04d      	beq.n	8000e70 <_printf_i+0x1b4>
 8000dd4:	4616      	mov	r6, r2
 8000dd6:	fbb5 f1f3 	udiv	r1, r5, r3
 8000dda:	fb03 5711 	mls	r7, r3, r1, r5
 8000dde:	5dc7      	ldrb	r7, [r0, r7]
 8000de0:	f806 7d01 	strb.w	r7, [r6, #-1]!
 8000de4:	462f      	mov	r7, r5
 8000de6:	42bb      	cmp	r3, r7
 8000de8:	460d      	mov	r5, r1
 8000dea:	d9f4      	bls.n	8000dd6 <_printf_i+0x11a>
 8000dec:	2b08      	cmp	r3, #8
 8000dee:	d10b      	bne.n	8000e08 <_printf_i+0x14c>
 8000df0:	6823      	ldr	r3, [r4, #0]
 8000df2:	07df      	lsls	r7, r3, #31
 8000df4:	d508      	bpl.n	8000e08 <_printf_i+0x14c>
 8000df6:	6923      	ldr	r3, [r4, #16]
 8000df8:	6861      	ldr	r1, [r4, #4]
 8000dfa:	4299      	cmp	r1, r3
 8000dfc:	bfde      	ittt	le
 8000dfe:	2330      	movle	r3, #48	; 0x30
 8000e00:	f806 3c01 	strble.w	r3, [r6, #-1]
 8000e04:	f106 36ff 	addle.w	r6, r6, #4294967295
 8000e08:	1b92      	subs	r2, r2, r6
 8000e0a:	6122      	str	r2, [r4, #16]
 8000e0c:	f8cd a000 	str.w	sl, [sp]
 8000e10:	464b      	mov	r3, r9
 8000e12:	aa03      	add	r2, sp, #12
 8000e14:	4621      	mov	r1, r4
 8000e16:	4640      	mov	r0, r8
 8000e18:	f7ff fee2 	bl	8000be0 <_printf_common>
 8000e1c:	3001      	adds	r0, #1
 8000e1e:	d14c      	bne.n	8000eba <_printf_i+0x1fe>
 8000e20:	f04f 30ff 	mov.w	r0, #4294967295
 8000e24:	b004      	add	sp, #16
 8000e26:	e8bd 87f0 	ldmia.w	sp!, {r4, r5, r6, r7, r8, r9, sl, pc}
 8000e2a:	4835      	ldr	r0, [pc, #212]	; (8000f00 <_printf_i+0x244>)
 8000e2c:	f884 7045 	strb.w	r7, [r4, #69]	; 0x45
 8000e30:	6823      	ldr	r3, [r4, #0]
 8000e32:	680e      	ldr	r6, [r1, #0]
 8000e34:	061f      	lsls	r7, r3, #24
 8000e36:	f856 5b04 	ldr.w	r5, [r6], #4
 8000e3a:	600e      	str	r6, [r1, #0]
 8000e3c:	d514      	bpl.n	8000e68 <_printf_i+0x1ac>
 8000e3e:	07d9      	lsls	r1, r3, #31
 8000e40:	bf44      	itt	mi
 8000e42:	f043 0320 	orrmi.w	r3, r3, #32
 8000e46:	6023      	strmi	r3, [r4, #0]
 8000e48:	b91d      	cbnz	r5, 8000e52 <_printf_i+0x196>
 8000e4a:	6823      	ldr	r3, [r4, #0]
 8000e4c:	f023 0320 	bic.w	r3, r3, #32
 8000e50:	6023      	str	r3, [r4, #0]
 8000e52:	2310      	movs	r3, #16
 8000e54:	e7b0      	b.n	8000db8 <_printf_i+0xfc>
 8000e56:	6823      	ldr	r3, [r4, #0]
 8000e58:	f043 0320 	orr.w	r3, r3, #32
 8000e5c:	6023      	str	r3, [r4, #0]
 8000e5e:	2378      	movs	r3, #120	; 0x78
 8000e60:	4828      	ldr	r0, [pc, #160]	; (8000f04 <_printf_i+0x248>)
 8000e62:	f884 3045 	strb.w	r3, [r4, #69]	; 0x45
 8000e66:	e7e3      	b.n	8000e30 <_printf_i+0x174>
 8000e68:	065e      	lsls	r6, r3, #25
 8000e6a:	bf48      	it	mi
 8000e6c:	b2ad      	uxthmi	r5, r5
 8000e6e:	e7e6      	b.n	8000e3e <_printf_i+0x182>
 8000e70:	4616      	mov	r6, r2
 8000e72:	e7bb      	b.n	8000dec <_printf_i+0x130>
 8000e74:	680b      	ldr	r3, [r1, #0]
 8000e76:	6826      	ldr	r6, [r4, #0]
 8000e78:	6960      	ldr	r0, [r4, #20]
 8000e7a:	1d1d      	adds	r5, r3, #4
 8000e7c:	600d      	str	r5, [r1, #0]
 8000e7e:	0635      	lsls	r5, r6, #24
 8000e80:	681b      	ldr	r3, [r3, #0]
 8000e82:	d501      	bpl.n	8000e88 <_printf_i+0x1cc>
 8000e84:	6018      	str	r0, [r3, #0]
 8000e86:	e002      	b.n	8000e8e <_printf_i+0x1d2>
 8000e88:	0671      	lsls	r1, r6, #25
 8000e8a:	d5fb      	bpl.n	8000e84 <_printf_i+0x1c8>
 8000e8c:	8018      	strh	r0, [r3, #0]
 8000e8e:	2300      	movs	r3, #0
 8000e90:	6123      	str	r3, [r4, #16]
 8000e92:	4616      	mov	r6, r2
 8000e94:	e7ba      	b.n	8000e0c <_printf_i+0x150>
 8000e96:	680b      	ldr	r3, [r1, #0]
 8000e98:	1d1a      	adds	r2, r3, #4
 8000e9a:	600a      	str	r2, [r1, #0]
 8000e9c:	681e      	ldr	r6, [r3, #0]
 8000e9e:	6862      	ldr	r2, [r4, #4]
 8000ea0:	2100      	movs	r1, #0
 8000ea2:	4630      	mov	r0, r6
 8000ea4:	f7ff f99c 	bl	80001e0 <memchr>
 8000ea8:	b108      	cbz	r0, 8000eae <_printf_i+0x1f2>
 8000eaa:	1b80      	subs	r0, r0, r6
 8000eac:	6060      	str	r0, [r4, #4]
 8000eae:	6863      	ldr	r3, [r4, #4]
 8000eb0:	6123      	str	r3, [r4, #16]
 8000eb2:	2300      	movs	r3, #0
 8000eb4:	f884 3043 	strb.w	r3, [r4, #67]	; 0x43
 8000eb8:	e7a8      	b.n	8000e0c <_printf_i+0x150>
 8000eba:	6923      	ldr	r3, [r4, #16]
 8000ebc:	4632      	mov	r2, r6
 8000ebe:	4649      	mov	r1, r9
 8000ec0:	4640      	mov	r0, r8
 8000ec2:	47d0      	blx	sl
 8000ec4:	3001      	adds	r0, #1
 8000ec6:	d0ab      	beq.n	8000e20 <_printf_i+0x164>
 8000ec8:	6823      	ldr	r3, [r4, #0]
 8000eca:	079b      	lsls	r3, r3, #30
 8000ecc:	d413      	bmi.n	8000ef6 <_printf_i+0x23a>
 8000ece:	68e0      	ldr	r0, [r4, #12]
 8000ed0:	9b03      	ldr	r3, [sp, #12]
 8000ed2:	4298      	cmp	r0, r3
 8000ed4:	bfb8      	it	lt
 8000ed6:	4618      	movlt	r0, r3
 8000ed8:	e7a4      	b.n	8000e24 <_printf_i+0x168>
 8000eda:	2301      	movs	r3, #1
 8000edc:	4632      	mov	r2, r6
 8000ede:	4649      	mov	r1, r9
 8000ee0:	4640      	mov	r0, r8
 8000ee2:	47d0      	blx	sl
 8000ee4:	3001      	adds	r0, #1
 8000ee6:	d09b      	beq.n	8000e20 <_printf_i+0x164>
 8000ee8:	3501      	adds	r5, #1
 8000eea:	68e3      	ldr	r3, [r4, #12]
 8000eec:	9903      	ldr	r1, [sp, #12]
 8000eee:	1a5b      	subs	r3, r3, r1
 8000ef0:	42ab      	cmp	r3, r5
 8000ef2:	dcf2      	bgt.n	8000eda <_printf_i+0x21e>
 8000ef4:	e7eb      	b.n	8000ece <_printf_i+0x212>
 8000ef6:	2500      	movs	r5, #0
 8000ef8:	f104 0619 	add.w	r6, r4, #25
 8000efc:	e7f5      	b.n	8000eea <_printf_i+0x22e>
 8000efe:	bf00      	nop
 8000f00:	080015a9 	.word	0x080015a9
 8000f04:	080015ba 	.word	0x080015ba

08000f08 <_sbrk_r>:
 8000f08:	b538      	push	{r3, r4, r5, lr}
 8000f0a:	4d06      	ldr	r5, [pc, #24]	; (8000f24 <_sbrk_r+0x1c>)
 8000f0c:	2300      	movs	r3, #0
 8000f0e:	4604      	mov	r4, r0
 8000f10:	4608      	mov	r0, r1
 8000f12:	602b      	str	r3, [r5, #0]
 8000f14:	f7ff fa4c 	bl	80003b0 <_sbrk>
 8000f18:	1c43      	adds	r3, r0, #1
 8000f1a:	d102      	bne.n	8000f22 <_sbrk_r+0x1a>
 8000f1c:	682b      	ldr	r3, [r5, #0]
 8000f1e:	b103      	cbz	r3, 8000f22 <_sbrk_r+0x1a>
 8000f20:	6023      	str	r3, [r4, #0]
 8000f22:	bd38      	pop	{r3, r4, r5, pc}
 8000f24:	20000098 	.word	0x20000098

08000f28 <__sread>:
 8000f28:	b510      	push	{r4, lr}
 8000f2a:	460c      	mov	r4, r1
 8000f2c:	f9b1 100e 	ldrsh.w	r1, [r1, #14]
 8000f30:	f000 fab4 	bl	800149c <_read_r>
 8000f34:	2800      	cmp	r0, #0
 8000f36:	bfab      	itete	ge
 8000f38:	6d63      	ldrge	r3, [r4, #84]	; 0x54
 8000f3a:	89a3      	ldrhlt	r3, [r4, #12]
 8000f3c:	181b      	addge	r3, r3, r0
 8000f3e:	f423 5380 	biclt.w	r3, r3, #4096	; 0x1000
 8000f42:	bfac      	ite	ge
 8000f44:	6563      	strge	r3, [r4, #84]	; 0x54
 8000f46:	81a3      	strhlt	r3, [r4, #12]
 8000f48:	bd10      	pop	{r4, pc}

08000f4a <__swrite>:
 8000f4a:	e92d 41f0 	stmdb	sp!, {r4, r5, r6, r7, r8, lr}
 8000f4e:	461f      	mov	r7, r3
 8000f50:	898b      	ldrh	r3, [r1, #12]
 8000f52:	05db      	lsls	r3, r3, #23
 8000f54:	4605      	mov	r5, r0
 8000f56:	460c      	mov	r4, r1
 8000f58:	4616      	mov	r6, r2
 8000f5a:	d505      	bpl.n	8000f68 <__swrite+0x1e>
 8000f5c:	f9b1 100e 	ldrsh.w	r1, [r1, #14]
 8000f60:	2302      	movs	r3, #2
 8000f62:	2200      	movs	r2, #0
 8000f64:	f000 f9c8 	bl	80012f8 <_lseek_r>
 8000f68:	89a3      	ldrh	r3, [r4, #12]
 8000f6a:	f9b4 100e 	ldrsh.w	r1, [r4, #14]
 8000f6e:	f423 5380 	bic.w	r3, r3, #4096	; 0x1000
 8000f72:	81a3      	strh	r3, [r4, #12]
 8000f74:	4632      	mov	r2, r6
 8000f76:	463b      	mov	r3, r7
 8000f78:	4628      	mov	r0, r5
 8000f7a:	e8bd 41f0 	ldmia.w	sp!, {r4, r5, r6, r7, r8, lr}
 8000f7e:	f000 b869 	b.w	8001054 <_write_r>

08000f82 <__sseek>:
 8000f82:	b510      	push	{r4, lr}
 8000f84:	460c      	mov	r4, r1
 8000f86:	f9b1 100e 	ldrsh.w	r1, [r1, #14]
 8000f8a:	f000 f9b5 	bl	80012f8 <_lseek_r>
 8000f8e:	1c43      	adds	r3, r0, #1
 8000f90:	89a3      	ldrh	r3, [r4, #12]
 8000f92:	bf15      	itete	ne
 8000f94:	6560      	strne	r0, [r4, #84]	; 0x54
 8000f96:	f423 5380 	biceq.w	r3, r3, #4096	; 0x1000
 8000f9a:	f443 5380 	orrne.w	r3, r3, #4096	; 0x1000
 8000f9e:	81a3      	strheq	r3, [r4, #12]
 8000fa0:	bf18      	it	ne
 8000fa2:	81a3      	strhne	r3, [r4, #12]
 8000fa4:	bd10      	pop	{r4, pc}

08000fa6 <__sclose>:
 8000fa6:	f9b1 100e 	ldrsh.w	r1, [r1, #14]
 8000faa:	f000 b8d3 	b.w	8001154 <_close_r>
	...

08000fb0 <__swbuf_r>:
 8000fb0:	b5f8      	push	{r3, r4, r5, r6, r7, lr}
 8000fb2:	460e      	mov	r6, r1
 8000fb4:	4614      	mov	r4, r2
 8000fb6:	4605      	mov	r5, r0
 8000fb8:	b118      	cbz	r0, 8000fc2 <__swbuf_r+0x12>
 8000fba:	6983      	ldr	r3, [r0, #24]
 8000fbc:	b90b      	cbnz	r3, 8000fc2 <__swbuf_r+0x12>
 8000fbe:	f7ff fbbb 	bl	8000738 <__sinit>
 8000fc2:	4b21      	ldr	r3, [pc, #132]	; (8001048 <__swbuf_r+0x98>)
 8000fc4:	429c      	cmp	r4, r3
 8000fc6:	d12b      	bne.n	8001020 <__swbuf_r+0x70>
 8000fc8:	686c      	ldr	r4, [r5, #4]
 8000fca:	69a3      	ldr	r3, [r4, #24]
 8000fcc:	60a3      	str	r3, [r4, #8]
 8000fce:	89a3      	ldrh	r3, [r4, #12]
 8000fd0:	071a      	lsls	r2, r3, #28
 8000fd2:	d52f      	bpl.n	8001034 <__swbuf_r+0x84>
 8000fd4:	6923      	ldr	r3, [r4, #16]
 8000fd6:	b36b      	cbz	r3, 8001034 <__swbuf_r+0x84>
 8000fd8:	6923      	ldr	r3, [r4, #16]
 8000fda:	6820      	ldr	r0, [r4, #0]
 8000fdc:	1ac0      	subs	r0, r0, r3
 8000fde:	6963      	ldr	r3, [r4, #20]
 8000fe0:	b2f6      	uxtb	r6, r6
 8000fe2:	4283      	cmp	r3, r0
 8000fe4:	4637      	mov	r7, r6
 8000fe6:	dc04      	bgt.n	8000ff2 <__swbuf_r+0x42>
 8000fe8:	4621      	mov	r1, r4
 8000fea:	4628      	mov	r0, r5
 8000fec:	f000 f948 	bl	8001280 <_fflush_r>
 8000ff0:	bb30      	cbnz	r0, 8001040 <__swbuf_r+0x90>
 8000ff2:	68a3      	ldr	r3, [r4, #8]
 8000ff4:	3b01      	subs	r3, #1
 8000ff6:	60a3      	str	r3, [r4, #8]
 8000ff8:	6823      	ldr	r3, [r4, #0]
 8000ffa:	1c5a      	adds	r2, r3, #1
 8000ffc:	6022      	str	r2, [r4, #0]
 8000ffe:	701e      	strb	r6, [r3, #0]
 8001000:	6963      	ldr	r3, [r4, #20]
 8001002:	3001      	adds	r0, #1
 8001004:	4283      	cmp	r3, r0
 8001006:	d004      	beq.n	8001012 <__swbuf_r+0x62>
 8001008:	89a3      	ldrh	r3, [r4, #12]
 800100a:	07db      	lsls	r3, r3, #31
 800100c:	d506      	bpl.n	800101c <__swbuf_r+0x6c>
 800100e:	2e0a      	cmp	r6, #10
 8001010:	d104      	bne.n	800101c <__swbuf_r+0x6c>
 8001012:	4621      	mov	r1, r4
 8001014:	4628      	mov	r0, r5
 8001016:	f000 f933 	bl	8001280 <_fflush_r>
 800101a:	b988      	cbnz	r0, 8001040 <__swbuf_r+0x90>
 800101c:	4638      	mov	r0, r7
 800101e:	bdf8      	pop	{r3, r4, r5, r6, r7, pc}
 8001020:	4b0a      	ldr	r3, [pc, #40]	; (800104c <__swbuf_r+0x9c>)
 8001022:	429c      	cmp	r4, r3
 8001024:	d101      	bne.n	800102a <__swbuf_r+0x7a>
 8001026:	68ac      	ldr	r4, [r5, #8]
 8001028:	e7cf      	b.n	8000fca <__swbuf_r+0x1a>
 800102a:	4b09      	ldr	r3, [pc, #36]	; (8001050 <__swbuf_r+0xa0>)
 800102c:	429c      	cmp	r4, r3
 800102e:	bf08      	it	eq
 8001030:	68ec      	ldreq	r4, [r5, #12]
 8001032:	e7ca      	b.n	8000fca <__swbuf_r+0x1a>
 8001034:	4621      	mov	r1, r4
 8001036:	4628      	mov	r0, r5
 8001038:	f000 f81e 	bl	8001078 <__swsetup_r>
 800103c:	2800      	cmp	r0, #0
 800103e:	d0cb      	beq.n	8000fd8 <__swbuf_r+0x28>
 8001040:	f04f 37ff 	mov.w	r7, #4294967295
 8001044:	e7ea      	b.n	800101c <__swbuf_r+0x6c>
 8001046:	bf00      	nop
 8001048:	08001558 	.word	0x08001558
 800104c:	08001578 	.word	0x08001578
 8001050:	08001538 	.word	0x08001538

08001054 <_write_r>:
 8001054:	b538      	push	{r3, r4, r5, lr}
 8001056:	4d07      	ldr	r5, [pc, #28]	; (8001074 <_write_r+0x20>)
 8001058:	4604      	mov	r4, r0
 800105a:	4608      	mov	r0, r1
 800105c:	4611      	mov	r1, r2
 800105e:	2200      	movs	r2, #0
 8001060:	602a      	str	r2, [r5, #0]
 8001062:	461a      	mov	r2, r3
 8001064:	f7ff f953 	bl	800030e <_write>
 8001068:	1c43      	adds	r3, r0, #1
 800106a:	d102      	bne.n	8001072 <_write_r+0x1e>
 800106c:	682b      	ldr	r3, [r5, #0]
 800106e:	b103      	cbz	r3, 8001072 <_write_r+0x1e>
 8001070:	6023      	str	r3, [r4, #0]
 8001072:	bd38      	pop	{r3, r4, r5, pc}
 8001074:	20000098 	.word	0x20000098

08001078 <__swsetup_r>:
 8001078:	4b32      	ldr	r3, [pc, #200]	; (8001144 <__swsetup_r+0xcc>)
 800107a:	b570      	push	{r4, r5, r6, lr}
 800107c:	681d      	ldr	r5, [r3, #0]
 800107e:	4606      	mov	r6, r0
 8001080:	460c      	mov	r4, r1
 8001082:	b125      	cbz	r5, 800108e <__swsetup_r+0x16>
 8001084:	69ab      	ldr	r3, [r5, #24]
 8001086:	b913      	cbnz	r3, 800108e <__swsetup_r+0x16>
 8001088:	4628      	mov	r0, r5
 800108a:	f7ff fb55 	bl	8000738 <__sinit>
 800108e:	4b2e      	ldr	r3, [pc, #184]	; (8001148 <__swsetup_r+0xd0>)
 8001090:	429c      	cmp	r4, r3
 8001092:	d10f      	bne.n	80010b4 <__swsetup_r+0x3c>
 8001094:	686c      	ldr	r4, [r5, #4]
 8001096:	89a3      	ldrh	r3, [r4, #12]
 8001098:	f9b4 200c 	ldrsh.w	r2, [r4, #12]
 800109c:	0719      	lsls	r1, r3, #28
 800109e:	d42c      	bmi.n	80010fa <__swsetup_r+0x82>
 80010a0:	06dd      	lsls	r5, r3, #27
 80010a2:	d411      	bmi.n	80010c8 <__swsetup_r+0x50>
 80010a4:	2309      	movs	r3, #9
 80010a6:	6033      	str	r3, [r6, #0]
 80010a8:	f042 0340 	orr.w	r3, r2, #64	; 0x40
 80010ac:	81a3      	strh	r3, [r4, #12]
 80010ae:	f04f 30ff 	mov.w	r0, #4294967295
 80010b2:	e03e      	b.n	8001132 <__swsetup_r+0xba>
 80010b4:	4b25      	ldr	r3, [pc, #148]	; (800114c <__swsetup_r+0xd4>)
 80010b6:	429c      	cmp	r4, r3
 80010b8:	d101      	bne.n	80010be <__swsetup_r+0x46>
 80010ba:	68ac      	ldr	r4, [r5, #8]
 80010bc:	e7eb      	b.n	8001096 <__swsetup_r+0x1e>
 80010be:	4b24      	ldr	r3, [pc, #144]	; (8001150 <__swsetup_r+0xd8>)
 80010c0:	429c      	cmp	r4, r3
 80010c2:	bf08      	it	eq
 80010c4:	68ec      	ldreq	r4, [r5, #12]
 80010c6:	e7e6      	b.n	8001096 <__swsetup_r+0x1e>
 80010c8:	0758      	lsls	r0, r3, #29
 80010ca:	d512      	bpl.n	80010f2 <__swsetup_r+0x7a>
 80010cc:	6b61      	ldr	r1, [r4, #52]	; 0x34
 80010ce:	b141      	cbz	r1, 80010e2 <__swsetup_r+0x6a>
 80010d0:	f104 0344 	add.w	r3, r4, #68	; 0x44
 80010d4:	4299      	cmp	r1, r3
 80010d6:	d002      	beq.n	80010de <__swsetup_r+0x66>
 80010d8:	4630      	mov	r0, r6
 80010da:	f000 f98f 	bl	80013fc <_free_r>
 80010de:	2300      	movs	r3, #0
 80010e0:	6363      	str	r3, [r4, #52]	; 0x34
 80010e2:	89a3      	ldrh	r3, [r4, #12]
 80010e4:	f023 0324 	bic.w	r3, r3, #36	; 0x24
 80010e8:	81a3      	strh	r3, [r4, #12]
 80010ea:	2300      	movs	r3, #0
 80010ec:	6063      	str	r3, [r4, #4]
 80010ee:	6923      	ldr	r3, [r4, #16]
 80010f0:	6023      	str	r3, [r4, #0]
 80010f2:	89a3      	ldrh	r3, [r4, #12]
 80010f4:	f043 0308 	orr.w	r3, r3, #8
 80010f8:	81a3      	strh	r3, [r4, #12]
 80010fa:	6923      	ldr	r3, [r4, #16]
 80010fc:	b94b      	cbnz	r3, 8001112 <__swsetup_r+0x9a>
 80010fe:	89a3      	ldrh	r3, [r4, #12]
 8001100:	f403 7320 	and.w	r3, r3, #640	; 0x280
 8001104:	f5b3 7f00 	cmp.w	r3, #512	; 0x200
 8001108:	d003      	beq.n	8001112 <__swsetup_r+0x9a>
 800110a:	4621      	mov	r1, r4
 800110c:	4630      	mov	r0, r6
 800110e:	f000 f929 	bl	8001364 <__smakebuf_r>
 8001112:	89a0      	ldrh	r0, [r4, #12]
 8001114:	f9b4 200c 	ldrsh.w	r2, [r4, #12]
 8001118:	f010 0301 	ands.w	r3, r0, #1
 800111c:	d00a      	beq.n	8001134 <__swsetup_r+0xbc>
 800111e:	2300      	movs	r3, #0
 8001120:	60a3      	str	r3, [r4, #8]
 8001122:	6963      	ldr	r3, [r4, #20]
 8001124:	425b      	negs	r3, r3
 8001126:	61a3      	str	r3, [r4, #24]
 8001128:	6923      	ldr	r3, [r4, #16]
 800112a:	b943      	cbnz	r3, 800113e <__swsetup_r+0xc6>
 800112c:	f010 0080 	ands.w	r0, r0, #128	; 0x80
 8001130:	d1ba      	bne.n	80010a8 <__swsetup_r+0x30>
 8001132:	bd70      	pop	{r4, r5, r6, pc}
 8001134:	0781      	lsls	r1, r0, #30
 8001136:	bf58      	it	pl
 8001138:	6963      	ldrpl	r3, [r4, #20]
 800113a:	60a3      	str	r3, [r4, #8]
 800113c:	e7f4      	b.n	8001128 <__swsetup_r+0xb0>
 800113e:	2000      	movs	r0, #0
 8001140:	e7f7      	b.n	8001132 <__swsetup_r+0xba>
 8001142:	bf00      	nop
 8001144:	20000000 	.word	0x20000000
 8001148:	08001558 	.word	0x08001558
 800114c:	08001578 	.word	0x08001578
 8001150:	08001538 	.word	0x08001538

08001154 <_close_r>:
 8001154:	b538      	push	{r3, r4, r5, lr}
 8001156:	4d06      	ldr	r5, [pc, #24]	; (8001170 <_close_r+0x1c>)
 8001158:	2300      	movs	r3, #0
 800115a:	4604      	mov	r4, r0
 800115c:	4608      	mov	r0, r1
 800115e:	602b      	str	r3, [r5, #0]
 8001160:	f7ff f8f1 	bl	8000346 <_close>
 8001164:	1c43      	adds	r3, r0, #1
 8001166:	d102      	bne.n	800116e <_close_r+0x1a>
 8001168:	682b      	ldr	r3, [r5, #0]
 800116a:	b103      	cbz	r3, 800116e <_close_r+0x1a>
 800116c:	6023      	str	r3, [r4, #0]
 800116e:	bd38      	pop	{r3, r4, r5, pc}
 8001170:	20000098 	.word	0x20000098

08001174 <__sflush_r>:
 8001174:	898a      	ldrh	r2, [r1, #12]
 8001176:	e92d 41f0 	stmdb	sp!, {r4, r5, r6, r7, r8, lr}
 800117a:	4605      	mov	r5, r0
 800117c:	0710      	lsls	r0, r2, #28
 800117e:	460c      	mov	r4, r1
 8001180:	d458      	bmi.n	8001234 <__sflush_r+0xc0>
 8001182:	684b      	ldr	r3, [r1, #4]
 8001184:	2b00      	cmp	r3, #0
 8001186:	dc05      	bgt.n	8001194 <__sflush_r+0x20>
 8001188:	6c0b      	ldr	r3, [r1, #64]	; 0x40
 800118a:	2b00      	cmp	r3, #0
 800118c:	dc02      	bgt.n	8001194 <__sflush_r+0x20>
 800118e:	2000      	movs	r0, #0
 8001190:	e8bd 81f0 	ldmia.w	sp!, {r4, r5, r6, r7, r8, pc}
 8001194:	6ae6      	ldr	r6, [r4, #44]	; 0x2c
 8001196:	2e00      	cmp	r6, #0
 8001198:	d0f9      	beq.n	800118e <__sflush_r+0x1a>
 800119a:	2300      	movs	r3, #0
 800119c:	f412 5280 	ands.w	r2, r2, #4096	; 0x1000
 80011a0:	682f      	ldr	r7, [r5, #0]
 80011a2:	602b      	str	r3, [r5, #0]
 80011a4:	d032      	beq.n	800120c <__sflush_r+0x98>
 80011a6:	6d60      	ldr	r0, [r4, #84]	; 0x54
 80011a8:	89a3      	ldrh	r3, [r4, #12]
 80011aa:	075a      	lsls	r2, r3, #29
 80011ac:	d505      	bpl.n	80011ba <__sflush_r+0x46>
 80011ae:	6863      	ldr	r3, [r4, #4]
 80011b0:	1ac0      	subs	r0, r0, r3
 80011b2:	6b63      	ldr	r3, [r4, #52]	; 0x34
 80011b4:	b10b      	cbz	r3, 80011ba <__sflush_r+0x46>
 80011b6:	6c23      	ldr	r3, [r4, #64]	; 0x40
 80011b8:	1ac0      	subs	r0, r0, r3
 80011ba:	2300      	movs	r3, #0
 80011bc:	4602      	mov	r2, r0
 80011be:	6ae6      	ldr	r6, [r4, #44]	; 0x2c
 80011c0:	6a21      	ldr	r1, [r4, #32]
 80011c2:	4628      	mov	r0, r5
 80011c4:	47b0      	blx	r6
 80011c6:	1c43      	adds	r3, r0, #1
 80011c8:	89a3      	ldrh	r3, [r4, #12]
 80011ca:	d106      	bne.n	80011da <__sflush_r+0x66>
 80011cc:	6829      	ldr	r1, [r5, #0]
 80011ce:	291d      	cmp	r1, #29
 80011d0:	d82c      	bhi.n	800122c <__sflush_r+0xb8>
 80011d2:	4a2a      	ldr	r2, [pc, #168]	; (800127c <__sflush_r+0x108>)
 80011d4:	40ca      	lsrs	r2, r1
 80011d6:	07d6      	lsls	r6, r2, #31
 80011d8:	d528      	bpl.n	800122c <__sflush_r+0xb8>
 80011da:	2200      	movs	r2, #0
 80011dc:	6062      	str	r2, [r4, #4]
 80011de:	04d9      	lsls	r1, r3, #19
 80011e0:	6922      	ldr	r2, [r4, #16]
 80011e2:	6022      	str	r2, [r4, #0]
 80011e4:	d504      	bpl.n	80011f0 <__sflush_r+0x7c>
 80011e6:	1c42      	adds	r2, r0, #1
 80011e8:	d101      	bne.n	80011ee <__sflush_r+0x7a>
 80011ea:	682b      	ldr	r3, [r5, #0]
 80011ec:	b903      	cbnz	r3, 80011f0 <__sflush_r+0x7c>
 80011ee:	6560      	str	r0, [r4, #84]	; 0x54
 80011f0:	6b61      	ldr	r1, [r4, #52]	; 0x34
 80011f2:	602f      	str	r7, [r5, #0]
 80011f4:	2900      	cmp	r1, #0
 80011f6:	d0ca      	beq.n	800118e <__sflush_r+0x1a>
 80011f8:	f104 0344 	add.w	r3, r4, #68	; 0x44
 80011fc:	4299      	cmp	r1, r3
 80011fe:	d002      	beq.n	8001206 <__sflush_r+0x92>
 8001200:	4628      	mov	r0, r5
 8001202:	f000 f8fb 	bl	80013fc <_free_r>
 8001206:	2000      	movs	r0, #0
 8001208:	6360      	str	r0, [r4, #52]	; 0x34
 800120a:	e7c1      	b.n	8001190 <__sflush_r+0x1c>
 800120c:	6a21      	ldr	r1, [r4, #32]
 800120e:	2301      	movs	r3, #1
 8001210:	4628      	mov	r0, r5
 8001212:	47b0      	blx	r6
 8001214:	1c41      	adds	r1, r0, #1
 8001216:	d1c7      	bne.n	80011a8 <__sflush_r+0x34>
 8001218:	682b      	ldr	r3, [r5, #0]
 800121a:	2b00      	cmp	r3, #0
 800121c:	d0c4      	beq.n	80011a8 <__sflush_r+0x34>
 800121e:	2b1d      	cmp	r3, #29
 8001220:	d001      	beq.n	8001226 <__sflush_r+0xb2>
 8001222:	2b16      	cmp	r3, #22
 8001224:	d101      	bne.n	800122a <__sflush_r+0xb6>
 8001226:	602f      	str	r7, [r5, #0]
 8001228:	e7b1      	b.n	800118e <__sflush_r+0x1a>
 800122a:	89a3      	ldrh	r3, [r4, #12]
 800122c:	f043 0340 	orr.w	r3, r3, #64	; 0x40
 8001230:	81a3      	strh	r3, [r4, #12]
 8001232:	e7ad      	b.n	8001190 <__sflush_r+0x1c>
 8001234:	690f      	ldr	r7, [r1, #16]
 8001236:	2f00      	cmp	r7, #0
 8001238:	d0a9      	beq.n	800118e <__sflush_r+0x1a>
 800123a:	0793      	lsls	r3, r2, #30
 800123c:	680e      	ldr	r6, [r1, #0]
 800123e:	bf08      	it	eq
 8001240:	694b      	ldreq	r3, [r1, #20]
 8001242:	600f      	str	r7, [r1, #0]
 8001244:	bf18      	it	ne
 8001246:	2300      	movne	r3, #0
 8001248:	eba6 0807 	sub.w	r8, r6, r7
 800124c:	608b      	str	r3, [r1, #8]
 800124e:	f1b8 0f00 	cmp.w	r8, #0
 8001252:	dd9c      	ble.n	800118e <__sflush_r+0x1a>
 8001254:	6a21      	ldr	r1, [r4, #32]
 8001256:	6aa6      	ldr	r6, [r4, #40]	; 0x28
 8001258:	4643      	mov	r3, r8
 800125a:	463a      	mov	r2, r7
 800125c:	4628      	mov	r0, r5
 800125e:	47b0      	blx	r6
 8001260:	2800      	cmp	r0, #0
 8001262:	dc06      	bgt.n	8001272 <__sflush_r+0xfe>
 8001264:	89a3      	ldrh	r3, [r4, #12]
 8001266:	f043 0340 	orr.w	r3, r3, #64	; 0x40
 800126a:	81a3      	strh	r3, [r4, #12]
 800126c:	f04f 30ff 	mov.w	r0, #4294967295
 8001270:	e78e      	b.n	8001190 <__sflush_r+0x1c>
 8001272:	4407      	add	r7, r0
 8001274:	eba8 0800 	sub.w	r8, r8, r0
 8001278:	e7e9      	b.n	800124e <__sflush_r+0xda>
 800127a:	bf00      	nop
 800127c:	20400001 	.word	0x20400001

08001280 <_fflush_r>:
 8001280:	b538      	push	{r3, r4, r5, lr}
 8001282:	690b      	ldr	r3, [r1, #16]
 8001284:	4605      	mov	r5, r0
 8001286:	460c      	mov	r4, r1
 8001288:	b913      	cbnz	r3, 8001290 <_fflush_r+0x10>
 800128a:	2500      	movs	r5, #0
 800128c:	4628      	mov	r0, r5
 800128e:	bd38      	pop	{r3, r4, r5, pc}
 8001290:	b118      	cbz	r0, 800129a <_fflush_r+0x1a>
 8001292:	6983      	ldr	r3, [r0, #24]
 8001294:	b90b      	cbnz	r3, 800129a <_fflush_r+0x1a>
 8001296:	f7ff fa4f 	bl	8000738 <__sinit>
 800129a:	4b14      	ldr	r3, [pc, #80]	; (80012ec <_fflush_r+0x6c>)
 800129c:	429c      	cmp	r4, r3
 800129e:	d11b      	bne.n	80012d8 <_fflush_r+0x58>
 80012a0:	686c      	ldr	r4, [r5, #4]
 80012a2:	f9b4 300c 	ldrsh.w	r3, [r4, #12]
 80012a6:	2b00      	cmp	r3, #0
 80012a8:	d0ef      	beq.n	800128a <_fflush_r+0xa>
 80012aa:	6e62      	ldr	r2, [r4, #100]	; 0x64
 80012ac:	07d0      	lsls	r0, r2, #31
 80012ae:	d404      	bmi.n	80012ba <_fflush_r+0x3a>
 80012b0:	0599      	lsls	r1, r3, #22
 80012b2:	d402      	bmi.n	80012ba <_fflush_r+0x3a>
 80012b4:	6da0      	ldr	r0, [r4, #88]	; 0x58
 80012b6:	f7ff fadd 	bl	8000874 <__retarget_lock_acquire_recursive>
 80012ba:	4628      	mov	r0, r5
 80012bc:	4621      	mov	r1, r4
 80012be:	f7ff ff59 	bl	8001174 <__sflush_r>
 80012c2:	6e63      	ldr	r3, [r4, #100]	; 0x64
 80012c4:	07da      	lsls	r2, r3, #31
 80012c6:	4605      	mov	r5, r0
 80012c8:	d4e0      	bmi.n	800128c <_fflush_r+0xc>
 80012ca:	89a3      	ldrh	r3, [r4, #12]
 80012cc:	059b      	lsls	r3, r3, #22
 80012ce:	d4dd      	bmi.n	800128c <_fflush_r+0xc>
 80012d0:	6da0      	ldr	r0, [r4, #88]	; 0x58
 80012d2:	f7ff fad0 	bl	8000876 <__retarget_lock_release_recursive>
 80012d6:	e7d9      	b.n	800128c <_fflush_r+0xc>
 80012d8:	4b05      	ldr	r3, [pc, #20]	; (80012f0 <_fflush_r+0x70>)
 80012da:	429c      	cmp	r4, r3
 80012dc:	d101      	bne.n	80012e2 <_fflush_r+0x62>
 80012de:	68ac      	ldr	r4, [r5, #8]
 80012e0:	e7df      	b.n	80012a2 <_fflush_r+0x22>
 80012e2:	4b04      	ldr	r3, [pc, #16]	; (80012f4 <_fflush_r+0x74>)
 80012e4:	429c      	cmp	r4, r3
 80012e6:	bf08      	it	eq
 80012e8:	68ec      	ldreq	r4, [r5, #12]
 80012ea:	e7da      	b.n	80012a2 <_fflush_r+0x22>
 80012ec:	08001558 	.word	0x08001558
 80012f0:	08001578 	.word	0x08001578
 80012f4:	08001538 	.word	0x08001538

080012f8 <_lseek_r>:
 80012f8:	b538      	push	{r3, r4, r5, lr}
 80012fa:	4d07      	ldr	r5, [pc, #28]	; (8001318 <_lseek_r+0x20>)
 80012fc:	4604      	mov	r4, r0
 80012fe:	4608      	mov	r0, r1
 8001300:	4611      	mov	r1, r2
 8001302:	2200      	movs	r2, #0
 8001304:	602a      	str	r2, [r5, #0]
 8001306:	461a      	mov	r2, r3
 8001308:	f7ff f844 	bl	8000394 <_lseek>
 800130c:	1c43      	adds	r3, r0, #1
 800130e:	d102      	bne.n	8001316 <_lseek_r+0x1e>
 8001310:	682b      	ldr	r3, [r5, #0]
 8001312:	b103      	cbz	r3, 8001316 <_lseek_r+0x1e>
 8001314:	6023      	str	r3, [r4, #0]
 8001316:	bd38      	pop	{r3, r4, r5, pc}
 8001318:	20000098 	.word	0x20000098

0800131c <__swhatbuf_r>:
 800131c:	b570      	push	{r4, r5, r6, lr}
 800131e:	460e      	mov	r6, r1
 8001320:	f9b1 100e 	ldrsh.w	r1, [r1, #14]
 8001324:	2900      	cmp	r1, #0
 8001326:	b096      	sub	sp, #88	; 0x58
 8001328:	4614      	mov	r4, r2
 800132a:	461d      	mov	r5, r3
 800132c:	da07      	bge.n	800133e <__swhatbuf_r+0x22>
 800132e:	2300      	movs	r3, #0
 8001330:	602b      	str	r3, [r5, #0]
 8001332:	89b3      	ldrh	r3, [r6, #12]
 8001334:	061a      	lsls	r2, r3, #24
 8001336:	d410      	bmi.n	800135a <__swhatbuf_r+0x3e>
 8001338:	f44f 6380 	mov.w	r3, #1024	; 0x400
 800133c:	e00e      	b.n	800135c <__swhatbuf_r+0x40>
 800133e:	466a      	mov	r2, sp
 8001340:	f000 f8be 	bl	80014c0 <_fstat_r>
 8001344:	2800      	cmp	r0, #0
 8001346:	dbf2      	blt.n	800132e <__swhatbuf_r+0x12>
 8001348:	9a01      	ldr	r2, [sp, #4]
 800134a:	f402 4270 	and.w	r2, r2, #61440	; 0xf000
 800134e:	f5a2 5300 	sub.w	r3, r2, #8192	; 0x2000
 8001352:	425a      	negs	r2, r3
 8001354:	415a      	adcs	r2, r3
 8001356:	602a      	str	r2, [r5, #0]
 8001358:	e7ee      	b.n	8001338 <__swhatbuf_r+0x1c>
 800135a:	2340      	movs	r3, #64	; 0x40
 800135c:	2000      	movs	r0, #0
 800135e:	6023      	str	r3, [r4, #0]
 8001360:	b016      	add	sp, #88	; 0x58
 8001362:	bd70      	pop	{r4, r5, r6, pc}

08001364 <__smakebuf_r>:
 8001364:	898b      	ldrh	r3, [r1, #12]
 8001366:	b573      	push	{r0, r1, r4, r5, r6, lr}
 8001368:	079d      	lsls	r5, r3, #30
 800136a:	4606      	mov	r6, r0
 800136c:	460c      	mov	r4, r1
 800136e:	d507      	bpl.n	8001380 <__smakebuf_r+0x1c>
 8001370:	f104 0347 	add.w	r3, r4, #71	; 0x47
 8001374:	6023      	str	r3, [r4, #0]
 8001376:	6123      	str	r3, [r4, #16]
 8001378:	2301      	movs	r3, #1
 800137a:	6163      	str	r3, [r4, #20]
 800137c:	b002      	add	sp, #8
 800137e:	bd70      	pop	{r4, r5, r6, pc}
 8001380:	ab01      	add	r3, sp, #4
 8001382:	466a      	mov	r2, sp
 8001384:	f7ff ffca 	bl	800131c <__swhatbuf_r>
 8001388:	9900      	ldr	r1, [sp, #0]
 800138a:	4605      	mov	r5, r0
 800138c:	4630      	mov	r0, r6
 800138e:	f7ff fa73 	bl	8000878 <_malloc_r>
 8001392:	b948      	cbnz	r0, 80013a8 <__smakebuf_r+0x44>
 8001394:	f9b4 300c 	ldrsh.w	r3, [r4, #12]
 8001398:	059a      	lsls	r2, r3, #22
 800139a:	d4ef      	bmi.n	800137c <__smakebuf_r+0x18>
 800139c:	f023 0303 	bic.w	r3, r3, #3
 80013a0:	f043 0302 	orr.w	r3, r3, #2
 80013a4:	81a3      	strh	r3, [r4, #12]
 80013a6:	e7e3      	b.n	8001370 <__smakebuf_r+0xc>
 80013a8:	4b0d      	ldr	r3, [pc, #52]	; (80013e0 <__smakebuf_r+0x7c>)
 80013aa:	62b3      	str	r3, [r6, #40]	; 0x28
 80013ac:	89a3      	ldrh	r3, [r4, #12]
 80013ae:	6020      	str	r0, [r4, #0]
 80013b0:	f043 0380 	orr.w	r3, r3, #128	; 0x80
 80013b4:	81a3      	strh	r3, [r4, #12]
 80013b6:	9b00      	ldr	r3, [sp, #0]
 80013b8:	6163      	str	r3, [r4, #20]
 80013ba:	9b01      	ldr	r3, [sp, #4]
 80013bc:	6120      	str	r0, [r4, #16]
 80013be:	b15b      	cbz	r3, 80013d8 <__smakebuf_r+0x74>
 80013c0:	f9b4 100e 	ldrsh.w	r1, [r4, #14]
 80013c4:	4630      	mov	r0, r6
 80013c6:	f000 f88d 	bl	80014e4 <_isatty_r>
 80013ca:	b128      	cbz	r0, 80013d8 <__smakebuf_r+0x74>
 80013cc:	89a3      	ldrh	r3, [r4, #12]
 80013ce:	f023 0303 	bic.w	r3, r3, #3
 80013d2:	f043 0301 	orr.w	r3, r3, #1
 80013d6:	81a3      	strh	r3, [r4, #12]
 80013d8:	89a0      	ldrh	r0, [r4, #12]
 80013da:	4305      	orrs	r5, r0
 80013dc:	81a5      	strh	r5, [r4, #12]
 80013de:	e7cd      	b.n	800137c <__smakebuf_r+0x18>
 80013e0:	080006d1 	.word	0x080006d1

080013e4 <__malloc_lock>:
 80013e4:	4801      	ldr	r0, [pc, #4]	; (80013ec <__malloc_lock+0x8>)
 80013e6:	f7ff ba45 	b.w	8000874 <__retarget_lock_acquire_recursive>
 80013ea:	bf00      	nop
 80013ec:	20000090 	.word	0x20000090

080013f0 <__malloc_unlock>:
 80013f0:	4801      	ldr	r0, [pc, #4]	; (80013f8 <__malloc_unlock+0x8>)
 80013f2:	f7ff ba40 	b.w	8000876 <__retarget_lock_release_recursive>
 80013f6:	bf00      	nop
 80013f8:	20000090 	.word	0x20000090

080013fc <_free_r>:
 80013fc:	b537      	push	{r0, r1, r2, r4, r5, lr}
 80013fe:	2900      	cmp	r1, #0
 8001400:	d048      	beq.n	8001494 <_free_r+0x98>
 8001402:	f851 3c04 	ldr.w	r3, [r1, #-4]
 8001406:	9001      	str	r0, [sp, #4]
 8001408:	2b00      	cmp	r3, #0
 800140a:	f1a1 0404 	sub.w	r4, r1, #4
 800140e:	bfb8      	it	lt
 8001410:	18e4      	addlt	r4, r4, r3
 8001412:	f7ff ffe7 	bl	80013e4 <__malloc_lock>
 8001416:	4a20      	ldr	r2, [pc, #128]	; (8001498 <_free_r+0x9c>)
 8001418:	9801      	ldr	r0, [sp, #4]
 800141a:	6813      	ldr	r3, [r2, #0]
 800141c:	4615      	mov	r5, r2
 800141e:	b933      	cbnz	r3, 800142e <_free_r+0x32>
 8001420:	6063      	str	r3, [r4, #4]
 8001422:	6014      	str	r4, [r2, #0]
 8001424:	b003      	add	sp, #12
 8001426:	e8bd 4030 	ldmia.w	sp!, {r4, r5, lr}
 800142a:	f7ff bfe1 	b.w	80013f0 <__malloc_unlock>
 800142e:	42a3      	cmp	r3, r4
 8001430:	d90b      	bls.n	800144a <_free_r+0x4e>
 8001432:	6821      	ldr	r1, [r4, #0]
 8001434:	1862      	adds	r2, r4, r1
 8001436:	4293      	cmp	r3, r2
 8001438:	bf04      	itt	eq
 800143a:	681a      	ldreq	r2, [r3, #0]
 800143c:	685b      	ldreq	r3, [r3, #4]
 800143e:	6063      	str	r3, [r4, #4]
 8001440:	bf04      	itt	eq
 8001442:	1852      	addeq	r2, r2, r1
 8001444:	6022      	streq	r2, [r4, #0]
 8001446:	602c      	str	r4, [r5, #0]
 8001448:	e7ec      	b.n	8001424 <_free_r+0x28>
 800144a:	461a      	mov	r2, r3
 800144c:	685b      	ldr	r3, [r3, #4]
 800144e:	b10b      	cbz	r3, 8001454 <_free_r+0x58>
 8001450:	42a3      	cmp	r3, r4
 8001452:	d9fa      	bls.n	800144a <_free_r+0x4e>
 8001454:	6811      	ldr	r1, [r2, #0]
 8001456:	1855      	adds	r5, r2, r1
 8001458:	42a5      	cmp	r5, r4
 800145a:	d10b      	bne.n	8001474 <_free_r+0x78>
 800145c:	6824      	ldr	r4, [r4, #0]
 800145e:	4421      	add	r1, r4
 8001460:	1854      	adds	r4, r2, r1
 8001462:	42a3      	cmp	r3, r4
 8001464:	6011      	str	r1, [r2, #0]
 8001466:	d1dd      	bne.n	8001424 <_free_r+0x28>
 8001468:	681c      	ldr	r4, [r3, #0]
 800146a:	685b      	ldr	r3, [r3, #4]
 800146c:	6053      	str	r3, [r2, #4]
 800146e:	4421      	add	r1, r4
 8001470:	6011      	str	r1, [r2, #0]
 8001472:	e7d7      	b.n	8001424 <_free_r+0x28>
 8001474:	d902      	bls.n	800147c <_free_r+0x80>
 8001476:	230c      	movs	r3, #12
 8001478:	6003      	str	r3, [r0, #0]
 800147a:	e7d3      	b.n	8001424 <_free_r+0x28>
 800147c:	6825      	ldr	r5, [r4, #0]
 800147e:	1961      	adds	r1, r4, r5
 8001480:	428b      	cmp	r3, r1
 8001482:	bf04      	itt	eq
 8001484:	6819      	ldreq	r1, [r3, #0]
 8001486:	685b      	ldreq	r3, [r3, #4]
 8001488:	6063      	str	r3, [r4, #4]
 800148a:	bf04      	itt	eq
 800148c:	1949      	addeq	r1, r1, r5
 800148e:	6021      	streq	r1, [r4, #0]
 8001490:	6054      	str	r4, [r2, #4]
 8001492:	e7c7      	b.n	8001424 <_free_r+0x28>
 8001494:	b003      	add	sp, #12
 8001496:	bd30      	pop	{r4, r5, pc}
 8001498:	20000084 	.word	0x20000084

0800149c <_read_r>:
 800149c:	b538      	push	{r3, r4, r5, lr}
 800149e:	4d07      	ldr	r5, [pc, #28]	; (80014bc <_read_r+0x20>)
 80014a0:	4604      	mov	r4, r0
 80014a2:	4608      	mov	r0, r1
 80014a4:	4611      	mov	r1, r2
 80014a6:	2200      	movs	r2, #0
 80014a8:	602a      	str	r2, [r5, #0]
 80014aa:	461a      	mov	r2, r3
 80014ac:	f7fe ff12 	bl	80002d4 <_read>
 80014b0:	1c43      	adds	r3, r0, #1
 80014b2:	d102      	bne.n	80014ba <_read_r+0x1e>
 80014b4:	682b      	ldr	r3, [r5, #0]
 80014b6:	b103      	cbz	r3, 80014ba <_read_r+0x1e>
 80014b8:	6023      	str	r3, [r4, #0]
 80014ba:	bd38      	pop	{r3, r4, r5, pc}
 80014bc:	20000098 	.word	0x20000098

080014c0 <_fstat_r>:
 80014c0:	b538      	push	{r3, r4, r5, lr}
 80014c2:	4d07      	ldr	r5, [pc, #28]	; (80014e0 <_fstat_r+0x20>)
 80014c4:	2300      	movs	r3, #0
 80014c6:	4604      	mov	r4, r0
 80014c8:	4608      	mov	r0, r1
 80014ca:	4611      	mov	r1, r2
 80014cc:	602b      	str	r3, [r5, #0]
 80014ce:	f7fe ff46 	bl	800035e <_fstat>
 80014d2:	1c43      	adds	r3, r0, #1
 80014d4:	d102      	bne.n	80014dc <_fstat_r+0x1c>
 80014d6:	682b      	ldr	r3, [r5, #0]
 80014d8:	b103      	cbz	r3, 80014dc <_fstat_r+0x1c>
 80014da:	6023      	str	r3, [r4, #0]
 80014dc:	bd38      	pop	{r3, r4, r5, pc}
 80014de:	bf00      	nop
 80014e0:	20000098 	.word	0x20000098

080014e4 <_isatty_r>:
 80014e4:	b538      	push	{r3, r4, r5, lr}
 80014e6:	4d06      	ldr	r5, [pc, #24]	; (8001500 <_isatty_r+0x1c>)
 80014e8:	2300      	movs	r3, #0
 80014ea:	4604      	mov	r4, r0
 80014ec:	4608      	mov	r0, r1
 80014ee:	602b      	str	r3, [r5, #0]
 80014f0:	f7fe ff45 	bl	800037e <_isatty>
 80014f4:	1c43      	adds	r3, r0, #1
 80014f6:	d102      	bne.n	80014fe <_isatty_r+0x1a>
 80014f8:	682b      	ldr	r3, [r5, #0]
 80014fa:	b103      	cbz	r3, 80014fe <_isatty_r+0x1a>
 80014fc:	6023      	str	r3, [r4, #0]
 80014fe:	bd38      	pop	{r3, r4, r5, pc}
 8001500:	20000098 	.word	0x20000098

08001504 <_init>:
 8001504:	b5f8      	push	{r3, r4, r5, r6, r7, lr}
 8001506:	bf00      	nop
 8001508:	bcf8      	pop	{r3, r4, r5, r6, r7}
 800150a:	bc08      	pop	{r3}
 800150c:	469e      	mov	lr, r3
 800150e:	4770      	bx	lr

08001510 <_fini>:
 8001510:	b5f8      	push	{r3, r4, r5, r6, r7, lr}
 8001512:	bf00      	nop
 8001514:	bcf8      	pop	{r3, r4, r5, r6, r7}
 8001516:	bc08      	pop	{r3}
 8001518:	469e      	mov	lr, r3
 800151a:	4770      	bx	lr
